ARM GAS  C:\Users\varun\AppData\Local\Temp\ccmQ1d3e.s 			page 1


   1              		.syntax unified
   2              		.cpu cortex-m0
   3              		.fpu softvfp
   4              		.eabi_attribute 20, 1
   5              		.eabi_attribute 21, 1
   6              		.eabi_attribute 23, 3
   7              		.eabi_attribute 24, 1
   8              		.eabi_attribute 25, 1
   9              		.eabi_attribute 26, 1
  10              		.eabi_attribute 30, 1
  11              		.eabi_attribute 34, 0
  12              		.eabi_attribute 18, 4
  13              		.thumb
  14              		.syntax unified
  15              		.file	"cyfitter_cfg.c"
  16              		.text
  17              	.Ltext0:
  18              		.cfi_sections	.debug_frame
  19              		.section	.text.cfg_write_bytes32,"ax",%progbits
  20              		.align	2
  21              		.code	16
  22              		.thumb_func
  23              		.type	cfg_write_bytes32, %function
  24              	cfg_write_bytes32:
  25              	.LFB3:
  26              		.file 1 "Generated_Source\\PSoC4\\cyfitter_cfg.c"
   1:Generated_Source\PSoC4/cyfitter_cfg.c **** 
   2:Generated_Source\PSoC4/cyfitter_cfg.c **** /*******************************************************************************
   3:Generated_Source\PSoC4/cyfitter_cfg.c **** * File Name: cyfitter_cfg.c
   4:Generated_Source\PSoC4/cyfitter_cfg.c **** * 
   5:Generated_Source\PSoC4/cyfitter_cfg.c **** * PSoC Creator  4.4
   6:Generated_Source\PSoC4/cyfitter_cfg.c **** *
   7:Generated_Source\PSoC4/cyfitter_cfg.c **** * Description:
   8:Generated_Source\PSoC4/cyfitter_cfg.c **** * This file contains device initialization code.
   9:Generated_Source\PSoC4/cyfitter_cfg.c **** * Except for the user defined sections in CyClockStartupError(), this file should not be modified.
  10:Generated_Source\PSoC4/cyfitter_cfg.c **** * This file is automatically generated by PSoC Creator.
  11:Generated_Source\PSoC4/cyfitter_cfg.c **** *
  12:Generated_Source\PSoC4/cyfitter_cfg.c **** ********************************************************************************
  13:Generated_Source\PSoC4/cyfitter_cfg.c **** * Copyright (c) 2007-2020 Cypress Semiconductor.  All rights reserved.
  14:Generated_Source\PSoC4/cyfitter_cfg.c **** * You may use this file only in accordance with the license, terms, conditions, 
  15:Generated_Source\PSoC4/cyfitter_cfg.c **** * disclaimers, and limitations in the end user license agreement accompanying 
  16:Generated_Source\PSoC4/cyfitter_cfg.c **** * the software package with which this file was provided.
  17:Generated_Source\PSoC4/cyfitter_cfg.c **** ********************************************************************************/
  18:Generated_Source\PSoC4/cyfitter_cfg.c **** 
  19:Generated_Source\PSoC4/cyfitter_cfg.c **** #include <string.h>
  20:Generated_Source\PSoC4/cyfitter_cfg.c **** #include "cytypes.h"
  21:Generated_Source\PSoC4/cyfitter_cfg.c **** #include "cydevice_trm.h"
  22:Generated_Source\PSoC4/cyfitter_cfg.c **** #include "cyfitter.h"
  23:Generated_Source\PSoC4/cyfitter_cfg.c **** #include "CyLib.h"
  24:Generated_Source\PSoC4/cyfitter_cfg.c **** #include "CyLFClk.h"
  25:Generated_Source\PSoC4/cyfitter_cfg.c **** #include "cyfitter_cfg.h"
  26:Generated_Source\PSoC4/cyfitter_cfg.c **** #include "cyapicallbacks.h"
  27:Generated_Source\PSoC4/cyfitter_cfg.c **** 
  28:Generated_Source\PSoC4/cyfitter_cfg.c **** 
  29:Generated_Source\PSoC4/cyfitter_cfg.c **** #if defined(__GNUC__) || defined(__ARMCC_VERSION)
  30:Generated_Source\PSoC4/cyfitter_cfg.c ****     #define CYPACKED 
  31:Generated_Source\PSoC4/cyfitter_cfg.c ****     #define CYPACKED_ATTR __attribute__ ((packed))
ARM GAS  C:\Users\varun\AppData\Local\Temp\ccmQ1d3e.s 			page 2


  32:Generated_Source\PSoC4/cyfitter_cfg.c ****     #define CYALIGNED __attribute__ ((aligned))
  33:Generated_Source\PSoC4/cyfitter_cfg.c ****     #define CY_CFG_UNUSED __attribute__ ((unused))
  34:Generated_Source\PSoC4/cyfitter_cfg.c ****     #ifndef CY_CFG_SECTION
  35:Generated_Source\PSoC4/cyfitter_cfg.c ****         #define CY_CFG_SECTION __attribute__ ((section(".psocinit")))
  36:Generated_Source\PSoC4/cyfitter_cfg.c ****     #endif
  37:Generated_Source\PSoC4/cyfitter_cfg.c ****     
  38:Generated_Source\PSoC4/cyfitter_cfg.c ****     #if defined(__ARMCC_VERSION)
  39:Generated_Source\PSoC4/cyfitter_cfg.c ****         #define CY_CFG_MEMORY_BARRIER() __memory_changed()
  40:Generated_Source\PSoC4/cyfitter_cfg.c ****     #else
  41:Generated_Source\PSoC4/cyfitter_cfg.c ****         #define CY_CFG_MEMORY_BARRIER() __sync_synchronize()
  42:Generated_Source\PSoC4/cyfitter_cfg.c ****     #endif
  43:Generated_Source\PSoC4/cyfitter_cfg.c ****     
  44:Generated_Source\PSoC4/cyfitter_cfg.c **** #elif defined(__ICCARM__)
  45:Generated_Source\PSoC4/cyfitter_cfg.c ****     #include <intrinsics.h>
  46:Generated_Source\PSoC4/cyfitter_cfg.c **** 
  47:Generated_Source\PSoC4/cyfitter_cfg.c ****     #define CYPACKED __packed
  48:Generated_Source\PSoC4/cyfitter_cfg.c ****     #define CYPACKED_ATTR 
  49:Generated_Source\PSoC4/cyfitter_cfg.c ****     #define CYALIGNED _Pragma("data_alignment=4")
  50:Generated_Source\PSoC4/cyfitter_cfg.c ****     #define CY_CFG_UNUSED _Pragma("diag_suppress=Pe177")
  51:Generated_Source\PSoC4/cyfitter_cfg.c ****     #define CY_CFG_SECTION _Pragma("location=\".psocinit\"")
  52:Generated_Source\PSoC4/cyfitter_cfg.c ****     
  53:Generated_Source\PSoC4/cyfitter_cfg.c ****     #define CY_CFG_MEMORY_BARRIER() __DMB()
  54:Generated_Source\PSoC4/cyfitter_cfg.c ****     
  55:Generated_Source\PSoC4/cyfitter_cfg.c **** #else
  56:Generated_Source\PSoC4/cyfitter_cfg.c ****     #error Unsupported toolchain
  57:Generated_Source\PSoC4/cyfitter_cfg.c **** #endif
  58:Generated_Source\PSoC4/cyfitter_cfg.c **** 
  59:Generated_Source\PSoC4/cyfitter_cfg.c **** #ifndef CYCODE
  60:Generated_Source\PSoC4/cyfitter_cfg.c ****     #define CYCODE
  61:Generated_Source\PSoC4/cyfitter_cfg.c **** #endif
  62:Generated_Source\PSoC4/cyfitter_cfg.c **** #ifndef CYDATA
  63:Generated_Source\PSoC4/cyfitter_cfg.c ****     #define CYDATA
  64:Generated_Source\PSoC4/cyfitter_cfg.c **** #endif
  65:Generated_Source\PSoC4/cyfitter_cfg.c **** #ifndef CYFAR
  66:Generated_Source\PSoC4/cyfitter_cfg.c ****     #define CYFAR
  67:Generated_Source\PSoC4/cyfitter_cfg.c **** #endif
  68:Generated_Source\PSoC4/cyfitter_cfg.c **** #ifndef CYXDATA
  69:Generated_Source\PSoC4/cyfitter_cfg.c ****     #define CYXDATA
  70:Generated_Source\PSoC4/cyfitter_cfg.c **** #endif
  71:Generated_Source\PSoC4/cyfitter_cfg.c **** 
  72:Generated_Source\PSoC4/cyfitter_cfg.c **** 
  73:Generated_Source\PSoC4/cyfitter_cfg.c **** CY_CFG_UNUSED
  74:Generated_Source\PSoC4/cyfitter_cfg.c **** static void CYMEMZERO(void *s, size_t n);
  75:Generated_Source\PSoC4/cyfitter_cfg.c **** CY_CFG_UNUSED
  76:Generated_Source\PSoC4/cyfitter_cfg.c **** static void CYMEMZERO(void *s, size_t n)
  77:Generated_Source\PSoC4/cyfitter_cfg.c **** {
  78:Generated_Source\PSoC4/cyfitter_cfg.c **** 	(void)memset(s, 0, n);
  79:Generated_Source\PSoC4/cyfitter_cfg.c **** }
  80:Generated_Source\PSoC4/cyfitter_cfg.c **** CY_CFG_UNUSED
  81:Generated_Source\PSoC4/cyfitter_cfg.c **** static void CYCONFIGCPY(void *dest, const void *src, size_t n);
  82:Generated_Source\PSoC4/cyfitter_cfg.c **** CY_CFG_UNUSED
  83:Generated_Source\PSoC4/cyfitter_cfg.c **** static void CYCONFIGCPY(void *dest, const void *src, size_t n)
  84:Generated_Source\PSoC4/cyfitter_cfg.c **** {
  85:Generated_Source\PSoC4/cyfitter_cfg.c **** 	(void)memcpy(dest, src, n);
  86:Generated_Source\PSoC4/cyfitter_cfg.c **** }
  87:Generated_Source\PSoC4/cyfitter_cfg.c **** CY_CFG_UNUSED
  88:Generated_Source\PSoC4/cyfitter_cfg.c **** static void CYCONFIGCPYCODE(void *dest, const void *src, size_t n);
ARM GAS  C:\Users\varun\AppData\Local\Temp\ccmQ1d3e.s 			page 3


  89:Generated_Source\PSoC4/cyfitter_cfg.c **** CY_CFG_UNUSED
  90:Generated_Source\PSoC4/cyfitter_cfg.c **** static void CYCONFIGCPYCODE(void *dest, const void *src, size_t n)
  91:Generated_Source\PSoC4/cyfitter_cfg.c **** {
  92:Generated_Source\PSoC4/cyfitter_cfg.c **** 	(void)memcpy(dest, src, n);
  93:Generated_Source\PSoC4/cyfitter_cfg.c **** }
  94:Generated_Source\PSoC4/cyfitter_cfg.c **** 
  95:Generated_Source\PSoC4/cyfitter_cfg.c **** 
  96:Generated_Source\PSoC4/cyfitter_cfg.c **** 
  97:Generated_Source\PSoC4/cyfitter_cfg.c **** 
  98:Generated_Source\PSoC4/cyfitter_cfg.c **** /* Clock startup error codes                                                   */
  99:Generated_Source\PSoC4/cyfitter_cfg.c **** #define CYCLOCKSTART_NO_ERROR    0u
 100:Generated_Source\PSoC4/cyfitter_cfg.c **** #define CYCLOCKSTART_XTAL_ERROR  1u
 101:Generated_Source\PSoC4/cyfitter_cfg.c **** #define CYCLOCKSTART_32KHZ_ERROR 2u
 102:Generated_Source\PSoC4/cyfitter_cfg.c **** #define CYCLOCKSTART_PLL_ERROR   3u
 103:Generated_Source\PSoC4/cyfitter_cfg.c **** #define CYCLOCKSTART_FLL_ERROR   4u
 104:Generated_Source\PSoC4/cyfitter_cfg.c **** #define CYCLOCKSTART_WCO_ERROR   5u
 105:Generated_Source\PSoC4/cyfitter_cfg.c **** 
 106:Generated_Source\PSoC4/cyfitter_cfg.c **** 
 107:Generated_Source\PSoC4/cyfitter_cfg.c **** #ifdef CY_NEED_CYCLOCKSTARTUPERROR
 108:Generated_Source\PSoC4/cyfitter_cfg.c **** /*******************************************************************************
 109:Generated_Source\PSoC4/cyfitter_cfg.c **** * Function Name: CyClockStartupError
 110:Generated_Source\PSoC4/cyfitter_cfg.c **** ********************************************************************************
 111:Generated_Source\PSoC4/cyfitter_cfg.c **** * Summary:
 112:Generated_Source\PSoC4/cyfitter_cfg.c **** *  If an error is encountered during clock configuration (crystal startup error,
 113:Generated_Source\PSoC4/cyfitter_cfg.c **** *  PLL lock error, etc.), the system will end up here.  Unless reimplemented by
 114:Generated_Source\PSoC4/cyfitter_cfg.c **** *  the customer, this function will stop in an infinite loop.
 115:Generated_Source\PSoC4/cyfitter_cfg.c **** *
 116:Generated_Source\PSoC4/cyfitter_cfg.c **** * Parameters:
 117:Generated_Source\PSoC4/cyfitter_cfg.c **** *   void
 118:Generated_Source\PSoC4/cyfitter_cfg.c **** *
 119:Generated_Source\PSoC4/cyfitter_cfg.c **** * Return:
 120:Generated_Source\PSoC4/cyfitter_cfg.c **** *   void
 121:Generated_Source\PSoC4/cyfitter_cfg.c **** *
 122:Generated_Source\PSoC4/cyfitter_cfg.c **** *******************************************************************************/
 123:Generated_Source\PSoC4/cyfitter_cfg.c **** CY_CFG_UNUSED
 124:Generated_Source\PSoC4/cyfitter_cfg.c **** static void CyClockStartupError(uint8 errorCode);
 125:Generated_Source\PSoC4/cyfitter_cfg.c **** CY_CFG_UNUSED
 126:Generated_Source\PSoC4/cyfitter_cfg.c **** static void CyClockStartupError(uint8 errorCode)
 127:Generated_Source\PSoC4/cyfitter_cfg.c **** {
 128:Generated_Source\PSoC4/cyfitter_cfg.c ****     /* To remove the compiler warning if errorCode not used.                */
 129:Generated_Source\PSoC4/cyfitter_cfg.c ****     errorCode = errorCode;
 130:Generated_Source\PSoC4/cyfitter_cfg.c **** 
 131:Generated_Source\PSoC4/cyfitter_cfg.c ****     /* If we have a clock startup error (bad MHz crystal, PLL lock, etc.),  */
 132:Generated_Source\PSoC4/cyfitter_cfg.c ****     /* we will end up here to allow the customer to implement something to  */
 133:Generated_Source\PSoC4/cyfitter_cfg.c ****     /* deal with the clock condition.                                       */
 134:Generated_Source\PSoC4/cyfitter_cfg.c **** 
 135:Generated_Source\PSoC4/cyfitter_cfg.c **** #ifdef CY_CFG_CLOCK_STARTUP_ERROR_CALLBACK
 136:Generated_Source\PSoC4/cyfitter_cfg.c ****     CY_CFG_Clock_Startup_ErrorCallback();
 137:Generated_Source\PSoC4/cyfitter_cfg.c **** #else
 138:Generated_Source\PSoC4/cyfitter_cfg.c ****     /*  If not using CY_CFG_CLOCK_STARTUP_ERROR_CALLBACK, place your clock startup code here. */
 139:Generated_Source\PSoC4/cyfitter_cfg.c ****     /* `#START CyClockStartupError` */
 140:Generated_Source\PSoC4/cyfitter_cfg.c **** 
 141:Generated_Source\PSoC4/cyfitter_cfg.c **** 
 142:Generated_Source\PSoC4/cyfitter_cfg.c **** 
 143:Generated_Source\PSoC4/cyfitter_cfg.c ****     /* `#END` */
 144:Generated_Source\PSoC4/cyfitter_cfg.c **** 
 145:Generated_Source\PSoC4/cyfitter_cfg.c ****     while(1) {}
ARM GAS  C:\Users\varun\AppData\Local\Temp\ccmQ1d3e.s 			page 4


 146:Generated_Source\PSoC4/cyfitter_cfg.c **** #endif /* CY_CFG_CLOCK_STARTUP_ERROR_CALLBACK */
 147:Generated_Source\PSoC4/cyfitter_cfg.c **** }
 148:Generated_Source\PSoC4/cyfitter_cfg.c **** #endif
 149:Generated_Source\PSoC4/cyfitter_cfg.c **** 
 150:Generated_Source\PSoC4/cyfitter_cfg.c **** #define CY_CFG_BASE_ADDR_COUNT 8u
 151:Generated_Source\PSoC4/cyfitter_cfg.c **** CYPACKED typedef struct
 152:Generated_Source\PSoC4/cyfitter_cfg.c **** {
 153:Generated_Source\PSoC4/cyfitter_cfg.c **** 	uint8 offset;
 154:Generated_Source\PSoC4/cyfitter_cfg.c **** 	uint8 value;
 155:Generated_Source\PSoC4/cyfitter_cfg.c **** } CYPACKED_ATTR cy_cfg_addrvalue_t;
 156:Generated_Source\PSoC4/cyfitter_cfg.c **** 
 157:Generated_Source\PSoC4/cyfitter_cfg.c **** 
 158:Generated_Source\PSoC4/cyfitter_cfg.c **** 
 159:Generated_Source\PSoC4/cyfitter_cfg.c **** /*******************************************************************************
 160:Generated_Source\PSoC4/cyfitter_cfg.c **** * Function Name: cfg_write_bytes32
 161:Generated_Source\PSoC4/cyfitter_cfg.c **** ********************************************************************************
 162:Generated_Source\PSoC4/cyfitter_cfg.c **** * Summary:
 163:Generated_Source\PSoC4/cyfitter_cfg.c **** *  This function is used for setting up the chip configuration areas that
 164:Generated_Source\PSoC4/cyfitter_cfg.c **** *  contain relatively sparse data.
 165:Generated_Source\PSoC4/cyfitter_cfg.c **** *
 166:Generated_Source\PSoC4/cyfitter_cfg.c **** * Parameters:
 167:Generated_Source\PSoC4/cyfitter_cfg.c **** *   void
 168:Generated_Source\PSoC4/cyfitter_cfg.c **** *
 169:Generated_Source\PSoC4/cyfitter_cfg.c **** * Return:
 170:Generated_Source\PSoC4/cyfitter_cfg.c **** *   void
 171:Generated_Source\PSoC4/cyfitter_cfg.c **** *
 172:Generated_Source\PSoC4/cyfitter_cfg.c **** *******************************************************************************/
 173:Generated_Source\PSoC4/cyfitter_cfg.c **** static void cfg_write_bytes32(const uint32 addr_table[], const cy_cfg_addrvalue_t data_table[]);
 174:Generated_Source\PSoC4/cyfitter_cfg.c **** static void cfg_write_bytes32(const uint32 addr_table[], const cy_cfg_addrvalue_t data_table[])
 175:Generated_Source\PSoC4/cyfitter_cfg.c **** {
  27              		.loc 1 175 0
  28              		.cfi_startproc
  29              		@ args = 0, pretend = 0, frame = 0
  30              		@ frame_needed = 0, uses_anonymous_args = 0
  31              	.LVL0:
  32 0000 F0B5     		push	{r4, r5, r6, r7, lr}
  33              		.cfi_def_cfa_offset 20
  34              		.cfi_offset 4, -20
  35              		.cfi_offset 5, -16
  36              		.cfi_offset 6, -12
  37              		.cfi_offset 7, -8
  38              		.cfi_offset 14, -4
  39              	.LVL1:
 176:Generated_Source\PSoC4/cyfitter_cfg.c **** 	/* For 32-bit little-endian architectures */
 177:Generated_Source\PSoC4/cyfitter_cfg.c **** 	uint32 i, j = 0u;
  40              		.loc 1 177 0
  41 0002 0025     		movs	r5, #0
 178:Generated_Source\PSoC4/cyfitter_cfg.c **** 	for (i = 0u; i < CY_CFG_BASE_ADDR_COUNT; i++)
  42              		.loc 1 178 0
  43 0004 0027     		movs	r7, #0
  44 0006 11E0     		b	.L2
  45              	.LVL2:
  46              	.L5:
  47              	.LBB2:
 179:Generated_Source\PSoC4/cyfitter_cfg.c **** 	{
 180:Generated_Source\PSoC4/cyfitter_cfg.c **** 		uint32 baseAddr = addr_table[i];
  48              		.loc 1 180 0
ARM GAS  C:\Users\varun\AppData\Local\Temp\ccmQ1d3e.s 			page 5


  49 0008 BB00     		lsls	r3, r7, #2
  50 000a C658     		ldr	r6, [r0, r3]
  51              	.LVL3:
 181:Generated_Source\PSoC4/cyfitter_cfg.c **** 		uint8 count = (uint8)baseAddr;
  52              		.loc 1 181 0
  53 000c F3B2     		uxtb	r3, r6
  54              	.LVL4:
 182:Generated_Source\PSoC4/cyfitter_cfg.c **** 		baseAddr &= 0xFFFFFF00u;
  55              		.loc 1 182 0
  56 000e FF22     		movs	r2, #255
  57 0010 9643     		bics	r6, r2
  58              	.LVL5:
 183:Generated_Source\PSoC4/cyfitter_cfg.c **** 		while (count != 0u)
  59              		.loc 1 183 0
  60 0012 08E0     		b	.L3
  61              	.L4:
 184:Generated_Source\PSoC4/cyfitter_cfg.c **** 		{
 185:Generated_Source\PSoC4/cyfitter_cfg.c **** 			CY_SET_REG8((void *)(baseAddr + data_table[j].offset), data_table[j].value);
  62              		.loc 1 185 0
  63 0014 6A00     		lsls	r2, r5, #1
  64 0016 8A18     		adds	r2, r1, r2
  65 0018 1478     		ldrb	r4, [r2]
  66 001a A419     		adds	r4, r4, r6
  67 001c 5278     		ldrb	r2, [r2, #1]
  68 001e 2270     		strb	r2, [r4]
 186:Generated_Source\PSoC4/cyfitter_cfg.c **** 			j++;
  69              		.loc 1 186 0
  70 0020 0135     		adds	r5, r5, #1
  71              	.LVL6:
 187:Generated_Source\PSoC4/cyfitter_cfg.c **** 			count--;
  72              		.loc 1 187 0
  73 0022 013B     		subs	r3, r3, #1
  74              	.LVL7:
  75 0024 DBB2     		uxtb	r3, r3
  76              	.LVL8:
  77              	.L3:
 183:Generated_Source\PSoC4/cyfitter_cfg.c **** 		{
  78              		.loc 1 183 0
  79 0026 002B     		cmp	r3, #0
  80 0028 F4D1     		bne	.L4
  81              	.LBE2:
 178:Generated_Source\PSoC4/cyfitter_cfg.c **** 	{
  82              		.loc 1 178 0 discriminator 2
  83 002a 0137     		adds	r7, r7, #1
  84              	.LVL9:
  85              	.L2:
 178:Generated_Source\PSoC4/cyfitter_cfg.c **** 	{
  86              		.loc 1 178 0 is_stmt 0 discriminator 1
  87 002c 072F     		cmp	r7, #7
  88 002e EBD9     		bls	.L5
 188:Generated_Source\PSoC4/cyfitter_cfg.c **** 		}
 189:Generated_Source\PSoC4/cyfitter_cfg.c **** 	}
 190:Generated_Source\PSoC4/cyfitter_cfg.c **** }
  89              		.loc 1 190 0 is_stmt 1
  90              		@ sp needed
  91              	.LVL10:
  92              	.LVL11:
ARM GAS  C:\Users\varun\AppData\Local\Temp\ccmQ1d3e.s 			page 6


  93 0030 F0BD     		pop	{r4, r5, r6, r7, pc}
  94              		.cfi_endproc
  95              	.LFE3:
  96              		.size	cfg_write_bytes32, .-cfg_write_bytes32
  97 0032 C046     		.section	.text.CYMEMZERO,"ax",%progbits
  98              		.align	2
  99              		.code	16
 100              		.thumb_func
 101              		.type	CYMEMZERO, %function
 102              	CYMEMZERO:
 103              	.LFB0:
  77:Generated_Source\PSoC4/cyfitter_cfg.c **** 	(void)memset(s, 0, n);
 104              		.loc 1 77 0
 105              		.cfi_startproc
 106              		@ args = 0, pretend = 0, frame = 0
 107              		@ frame_needed = 0, uses_anonymous_args = 0
 108              	.LVL12:
 109 0000 10B5     		push	{r4, lr}
 110              		.cfi_def_cfa_offset 8
 111              		.cfi_offset 4, -8
 112              		.cfi_offset 14, -4
 113 0002 0A00     		movs	r2, r1
  78:Generated_Source\PSoC4/cyfitter_cfg.c **** }
 114              		.loc 1 78 0
 115 0004 0021     		movs	r1, #0
 116              	.LVL13:
 117 0006 FFF7FEFF 		bl	memset
 118              	.LVL14:
  79:Generated_Source\PSoC4/cyfitter_cfg.c **** CY_CFG_UNUSED
 119              		.loc 1 79 0
 120              		@ sp needed
 121 000a 10BD     		pop	{r4, pc}
 122              		.cfi_endproc
 123              	.LFE0:
 124              		.size	CYMEMZERO, .-CYMEMZERO
 125              		.section	.psocinit,"ax",%progbits
 126              		.align	2
 127              		.code	16
 128              		.thumb_func
 129              		.type	ClockSetup, %function
 130              	ClockSetup:
 131              	.LFB4:
 191:Generated_Source\PSoC4/cyfitter_cfg.c **** 
 192:Generated_Source\PSoC4/cyfitter_cfg.c **** 
 193:Generated_Source\PSoC4/cyfitter_cfg.c **** /*******************************************************************************
 194:Generated_Source\PSoC4/cyfitter_cfg.c **** * Function Name: ClockSetup
 195:Generated_Source\PSoC4/cyfitter_cfg.c **** ********************************************************************************
 196:Generated_Source\PSoC4/cyfitter_cfg.c **** *
 197:Generated_Source\PSoC4/cyfitter_cfg.c **** * Summary:
 198:Generated_Source\PSoC4/cyfitter_cfg.c **** *   Performs the initialization of all of the clocks in the device based on the
 199:Generated_Source\PSoC4/cyfitter_cfg.c **** *   settings in the Clock tab of the DWR.  This includes enabling the requested
 200:Generated_Source\PSoC4/cyfitter_cfg.c **** *   clocks and setting the necessary dividers to produce the desired frequency. 
 201:Generated_Source\PSoC4/cyfitter_cfg.c **** *
 202:Generated_Source\PSoC4/cyfitter_cfg.c **** * Parameters:
 203:Generated_Source\PSoC4/cyfitter_cfg.c **** *   void
 204:Generated_Source\PSoC4/cyfitter_cfg.c **** *
 205:Generated_Source\PSoC4/cyfitter_cfg.c **** * Return:
ARM GAS  C:\Users\varun\AppData\Local\Temp\ccmQ1d3e.s 			page 7


 206:Generated_Source\PSoC4/cyfitter_cfg.c **** *   void
 207:Generated_Source\PSoC4/cyfitter_cfg.c **** *
 208:Generated_Source\PSoC4/cyfitter_cfg.c **** *******************************************************************************/
 209:Generated_Source\PSoC4/cyfitter_cfg.c **** static void ClockSetup(void);
 210:Generated_Source\PSoC4/cyfitter_cfg.c **** CY_CFG_SECTION
 211:Generated_Source\PSoC4/cyfitter_cfg.c **** static void ClockSetup(void)
 212:Generated_Source\PSoC4/cyfitter_cfg.c **** {
 132              		.loc 1 212 0
 133              		.cfi_startproc
 134              		@ args = 0, pretend = 0, frame = 0
 135              		@ frame_needed = 0, uses_anonymous_args = 0
 136 0000 70B5     		push	{r4, r5, r6, lr}
 137              		.cfi_def_cfa_offset 16
 138              		.cfi_offset 4, -16
 139              		.cfi_offset 5, -12
 140              		.cfi_offset 6, -8
 141              		.cfi_offset 14, -4
 213:Generated_Source\PSoC4/cyfitter_cfg.c **** 	/* Enable HALF_EN before trimming for the flash accelerator. */
 214:Generated_Source\PSoC4/cyfitter_cfg.c **** 	CY_SET_REG32((void CYXDATA *)(CYREG_CLK_SELECT), (CY_GET_REG32((void *)CYREG_CLK_SELECT) | 0x00040
 142              		.loc 1 214 0
 143 0002 194C     		ldr	r4, .L8
 144 0004 2368     		ldr	r3, [r4]
 145 0006 8022     		movs	r2, #128
 146 0008 D202     		lsls	r2, r2, #11
 147 000a 1343     		orrs	r3, r2
 148 000c 2360     		str	r3, [r4]
 215:Generated_Source\PSoC4/cyfitter_cfg.c **** 
 216:Generated_Source\PSoC4/cyfitter_cfg.c **** 	/* Setup and trim IMO based on desired frequency. */
 217:Generated_Source\PSoC4/cyfitter_cfg.c **** 	CySysClkWriteImoFreq(24u);
 149              		.loc 1 217 0
 150 000e 1820     		movs	r0, #24
 151 0010 FFF7FEFF 		bl	CySysClkWriteImoFreq
 152              	.LVL15:
 218:Generated_Source\PSoC4/cyfitter_cfg.c **** 
 219:Generated_Source\PSoC4/cyfitter_cfg.c **** 	/* Disable HALF_EN since it is not required at this IMO frequency. */
 220:Generated_Source\PSoC4/cyfitter_cfg.c **** 	CY_SET_REG32((void CYXDATA *)(CYREG_CLK_SELECT), (CY_GET_REG32((void *)CYREG_CLK_SELECT) & 0xFFFBF
 153              		.loc 1 220 0
 154 0014 2268     		ldr	r2, [r4]
 155 0016 154B     		ldr	r3, .L8+4
 156 0018 1340     		ands	r3, r2
 157 001a 2360     		str	r3, [r4]
 221:Generated_Source\PSoC4/cyfitter_cfg.c **** 	/* CYDEV_CLK_ILO_CONFIG Starting address: CYDEV_CLK_ILO_CONFIG */
 222:Generated_Source\PSoC4/cyfitter_cfg.c **** 	CY_SET_REG32((void *)(CYREG_CLK_ILO_CONFIG), 0x80000006u);
 158              		.loc 1 222 0
 159 001c 144A     		ldr	r2, .L8+8
 160 001e 154B     		ldr	r3, .L8+12
 161 0020 1A60     		str	r2, [r3]
 223:Generated_Source\PSoC4/cyfitter_cfg.c **** 
 224:Generated_Source\PSoC4/cyfitter_cfg.c **** 
 225:Generated_Source\PSoC4/cyfitter_cfg.c **** 	/* CYDEV_CLK_SELECT00 Starting address: CYDEV_CLK_SELECT00 */
 226:Generated_Source\PSoC4/cyfitter_cfg.c **** 	CY_SET_REG32((void *)(CYREG_CLK_SELECT02), 0x00000020u);
 162              		.loc 1 226 0
 163 0022 2022     		movs	r2, #32
 164 0024 144B     		ldr	r3, .L8+16
 165 0026 1A60     		str	r2, [r3]
 227:Generated_Source\PSoC4/cyfitter_cfg.c **** 	CY_SET_REG32((void *)(CYREG_CLK_SELECT07), 0x00000030u);
 166              		.loc 1 227 0
ARM GAS  C:\Users\varun\AppData\Local\Temp\ccmQ1d3e.s 			page 8


 167 0028 1032     		adds	r2, r2, #16
 168 002a 144B     		ldr	r3, .L8+20
 169 002c 1A60     		str	r2, [r3]
 228:Generated_Source\PSoC4/cyfitter_cfg.c **** 	CY_SET_REG32((void *)(CYREG_CLK_SELECT12), 0x00000010u);
 170              		.loc 1 228 0
 171 002e 203A     		subs	r2, r2, #32
 172 0030 134B     		ldr	r3, .L8+24
 173 0032 1A60     		str	r2, [r3]
 229:Generated_Source\PSoC4/cyfitter_cfg.c **** 
 230:Generated_Source\PSoC4/cyfitter_cfg.c **** 	/* CYDEV_CLK_IMO_CONFIG Starting address: CYDEV_CLK_IMO_CONFIG */
 231:Generated_Source\PSoC4/cyfitter_cfg.c **** 	CY_SET_REG32((void *)(CYREG_CLK_IMO_CONFIG), 0x82000000u);
 174              		.loc 1 231 0
 175 0034 8222     		movs	r2, #130
 176 0036 1206     		lsls	r2, r2, #24
 177 0038 124B     		ldr	r3, .L8+28
 178 003a 1A60     		str	r2, [r3]
 232:Generated_Source\PSoC4/cyfitter_cfg.c **** 
 233:Generated_Source\PSoC4/cyfitter_cfg.c **** 	/* CYDEV_CLK_SELECT Starting address: CYDEV_CLK_SELECT */
 234:Generated_Source\PSoC4/cyfitter_cfg.c **** 	CY_SET_REG32((void *)(CYREG_CLK_SELECT), 0x00000000u);
 179              		.loc 1 234 0
 180 003c 0025     		movs	r5, #0
 181 003e 2560     		str	r5, [r4]
 235:Generated_Source\PSoC4/cyfitter_cfg.c **** 
 236:Generated_Source\PSoC4/cyfitter_cfg.c **** 	/* CYDEV_CLK_DIVIDER_A00 Starting address: CYDEV_CLK_DIVIDER_A00 */
 237:Generated_Source\PSoC4/cyfitter_cfg.c **** 	CY_SET_REG32((void *)(CYREG_CLK_DIVIDER_A00), 0x80000001u);
 182              		.loc 1 237 0
 183 0040 114A     		ldr	r2, .L8+32
 184 0042 124B     		ldr	r3, .L8+36
 185 0044 1A60     		str	r2, [r3]
 238:Generated_Source\PSoC4/cyfitter_cfg.c **** 
 239:Generated_Source\PSoC4/cyfitter_cfg.c **** 	/* CYDEV_CLK_DIVIDER_B00 Starting address: CYDEV_CLK_DIVIDER_B00 */
 240:Generated_Source\PSoC4/cyfitter_cfg.c **** 	CY_SET_REG32((void *)(CYREG_CLK_DIVIDER_B00), 0x80000002u);
 186              		.loc 1 240 0
 187 0046 124A     		ldr	r2, .L8+40
 188 0048 124B     		ldr	r3, .L8+44
 189 004a 1A60     		str	r2, [r3]
 241:Generated_Source\PSoC4/cyfitter_cfg.c **** 
 242:Generated_Source\PSoC4/cyfitter_cfg.c **** 	/* CYDEV_CLK_DIVIDER_C00 Starting address: CYDEV_CLK_DIVIDER_C00 */
 243:Generated_Source\PSoC4/cyfitter_cfg.c **** 	CY_SET_REG32((void *)(CYREG_CLK_DIVIDER_C00), 0x8000000Fu);
 190              		.loc 1 243 0
 191 004c 124A     		ldr	r2, .L8+48
 192 004e 134B     		ldr	r3, .L8+52
 193 0050 1A60     		str	r2, [r3]
 244:Generated_Source\PSoC4/cyfitter_cfg.c **** 
 245:Generated_Source\PSoC4/cyfitter_cfg.c **** 	(void)CyIntSetVector(9u, &CySysWdtIsr);
 194              		.loc 1 245 0
 195 0052 1349     		ldr	r1, .L8+56
 196 0054 0920     		movs	r0, #9
 197 0056 FFF7FEFF 		bl	CyIntSetVector
 198              	.LVL16:
 246:Generated_Source\PSoC4/cyfitter_cfg.c **** 	CyIntEnable(9u);
 199              		.loc 1 246 0
 200 005a 0920     		movs	r0, #9
 201 005c FFF7FEFF 		bl	CyIntEnable
 202              	.LVL17:
 247:Generated_Source\PSoC4/cyfitter_cfg.c **** 	CY_SET_REG32((void *)(CYREG_WDT_CONFIG), 0x00000000u);
 203              		.loc 1 247 0
ARM GAS  C:\Users\varun\AppData\Local\Temp\ccmQ1d3e.s 			page 9


 204 0060 104B     		ldr	r3, .L8+60
 205 0062 1D60     		str	r5, [r3]
 248:Generated_Source\PSoC4/cyfitter_cfg.c **** }
 206              		.loc 1 248 0
 207              		@ sp needed
 208 0064 70BD     		pop	{r4, r5, r6, pc}
 209              	.L9:
 210 0066 C046     		.align	2
 211              	.L8:
 212 0068 00010B40 		.word	1074462976
 213 006c FFFFFBFF 		.word	-262145
 214 0070 06000080 		.word	-2147483642
 215 0074 04010B40 		.word	1074462980
 216 0078 08020240 		.word	1073873416
 217 007c 1C020240 		.word	1073873436
 218 0080 30020240 		.word	1073873456
 219 0084 08010B40 		.word	1074462984
 220 0088 01000080 		.word	-2147483647
 221 008c 00000240 		.word	1073872896
 222 0090 02000080 		.word	-2147483646
 223 0094 40000240 		.word	1073872960
 224 0098 0F000080 		.word	-2147483633
 225 009c 80000240 		.word	1073873024
 226 00a0 00000000 		.word	CySysWdtIsr
 227 00a4 0C020B40 		.word	1074463244
 228              		.cfi_endproc
 229              	.LFE4:
 230              		.size	ClockSetup, .-ClockSetup
 231              		.section	.text.SetAnalogRoutingPumps,"ax",%progbits
 232              		.align	2
 233              		.global	SetAnalogRoutingPumps
 234              		.code	16
 235              		.thumb_func
 236              		.type	SetAnalogRoutingPumps, %function
 237              	SetAnalogRoutingPumps:
 238              	.LFB6:
 249:Generated_Source\PSoC4/cyfitter_cfg.c **** 
 250:Generated_Source\PSoC4/cyfitter_cfg.c **** 
 251:Generated_Source\PSoC4/cyfitter_cfg.c **** /* Analog API Functions */
 252:Generated_Source\PSoC4/cyfitter_cfg.c **** 
 253:Generated_Source\PSoC4/cyfitter_cfg.c **** 
 254:Generated_Source\PSoC4/cyfitter_cfg.c **** /*******************************************************************************
 255:Generated_Source\PSoC4/cyfitter_cfg.c **** * Function Name: AnalogSetDefault
 256:Generated_Source\PSoC4/cyfitter_cfg.c **** ********************************************************************************
 257:Generated_Source\PSoC4/cyfitter_cfg.c **** *
 258:Generated_Source\PSoC4/cyfitter_cfg.c **** * Summary:
 259:Generated_Source\PSoC4/cyfitter_cfg.c **** *  Sets up the analog portions of the chip to default values based on chip
 260:Generated_Source\PSoC4/cyfitter_cfg.c **** *  configuration options from the project.
 261:Generated_Source\PSoC4/cyfitter_cfg.c **** *
 262:Generated_Source\PSoC4/cyfitter_cfg.c **** * Parameters:
 263:Generated_Source\PSoC4/cyfitter_cfg.c **** *  void
 264:Generated_Source\PSoC4/cyfitter_cfg.c **** *
 265:Generated_Source\PSoC4/cyfitter_cfg.c **** * Return:
 266:Generated_Source\PSoC4/cyfitter_cfg.c **** *  void
 267:Generated_Source\PSoC4/cyfitter_cfg.c **** *
 268:Generated_Source\PSoC4/cyfitter_cfg.c **** *******************************************************************************/
 269:Generated_Source\PSoC4/cyfitter_cfg.c **** static void AnalogSetDefault(void);
ARM GAS  C:\Users\varun\AppData\Local\Temp\ccmQ1d3e.s 			page 10


 270:Generated_Source\PSoC4/cyfitter_cfg.c **** static void AnalogSetDefault(void)
 271:Generated_Source\PSoC4/cyfitter_cfg.c **** {
 272:Generated_Source\PSoC4/cyfitter_cfg.c **** 	CY_SET_XTND_REG32((void CYFAR *)CYREG_SAR_MUX_SWITCH0, 0x00040000u);
 273:Generated_Source\PSoC4/cyfitter_cfg.c **** 	SetAnalogRoutingPumps(1);
 274:Generated_Source\PSoC4/cyfitter_cfg.c **** }
 275:Generated_Source\PSoC4/cyfitter_cfg.c **** 
 276:Generated_Source\PSoC4/cyfitter_cfg.c **** 
 277:Generated_Source\PSoC4/cyfitter_cfg.c **** /*******************************************************************************
 278:Generated_Source\PSoC4/cyfitter_cfg.c **** * Function Name: SetAnalogRoutingPumps
 279:Generated_Source\PSoC4/cyfitter_cfg.c **** ********************************************************************************
 280:Generated_Source\PSoC4/cyfitter_cfg.c **** *
 281:Generated_Source\PSoC4/cyfitter_cfg.c **** * Summary:
 282:Generated_Source\PSoC4/cyfitter_cfg.c **** * Enables or disables the analog pumps feeding analog routing switches.
 283:Generated_Source\PSoC4/cyfitter_cfg.c **** * Intended to be called at startup, based on the Vdda system configuration;
 284:Generated_Source\PSoC4/cyfitter_cfg.c **** * may be called during operation when the user informs us that the Vdda voltage crossed the pump th
 285:Generated_Source\PSoC4/cyfitter_cfg.c **** *
 286:Generated_Source\PSoC4/cyfitter_cfg.c **** * Parameters:
 287:Generated_Source\PSoC4/cyfitter_cfg.c **** *  enabled - 1 to enable the pumps, 0 to disable the pumps
 288:Generated_Source\PSoC4/cyfitter_cfg.c **** *
 289:Generated_Source\PSoC4/cyfitter_cfg.c **** * Return:
 290:Generated_Source\PSoC4/cyfitter_cfg.c **** *  void
 291:Generated_Source\PSoC4/cyfitter_cfg.c **** *
 292:Generated_Source\PSoC4/cyfitter_cfg.c **** *******************************************************************************/
 293:Generated_Source\PSoC4/cyfitter_cfg.c **** void SetAnalogRoutingPumps(uint8 enabled)
 294:Generated_Source\PSoC4/cyfitter_cfg.c **** {
 239              		.loc 1 294 0
 240              		.cfi_startproc
 241              		@ args = 0, pretend = 0, frame = 0
 242              		@ frame_needed = 0, uses_anonymous_args = 0
 243              		@ link register save eliminated.
 244              	.LVL18:
 295:Generated_Source\PSoC4/cyfitter_cfg.c **** 	uint32 regValue = CY_GET_XTND_REG32((void *)(CYREG_SAR_PUMP_CTRL));
 245              		.loc 1 295 0
 246 0000 064B     		ldr	r3, .L13
 247 0002 1B68     		ldr	r3, [r3]
 248              	.LVL19:
 296:Generated_Source\PSoC4/cyfitter_cfg.c **** 	if (enabled != 0u)
 249              		.loc 1 296 0
 250 0004 0028     		cmp	r0, #0
 251 0006 03D0     		beq	.L11
 297:Generated_Source\PSoC4/cyfitter_cfg.c **** 	{
 298:Generated_Source\PSoC4/cyfitter_cfg.c **** 		regValue |= 0x80000000u;
 252              		.loc 1 298 0
 253 0008 8022     		movs	r2, #128
 254 000a 1206     		lsls	r2, r2, #24
 255 000c 1343     		orrs	r3, r2
 256              	.LVL20:
 257 000e 01E0     		b	.L12
 258              	.L11:
 299:Generated_Source\PSoC4/cyfitter_cfg.c **** 	}
 300:Generated_Source\PSoC4/cyfitter_cfg.c **** 	else
 301:Generated_Source\PSoC4/cyfitter_cfg.c **** 	{
 302:Generated_Source\PSoC4/cyfitter_cfg.c **** 		regValue &= ~0x80000000u;
 259              		.loc 1 302 0
 260 0010 5B00     		lsls	r3, r3, #1
 261              	.LVL21:
 262 0012 5B08     		lsrs	r3, r3, #1
ARM GAS  C:\Users\varun\AppData\Local\Temp\ccmQ1d3e.s 			page 11


 263              	.LVL22:
 264              	.L12:
 303:Generated_Source\PSoC4/cyfitter_cfg.c **** 	}
 304:Generated_Source\PSoC4/cyfitter_cfg.c **** 	CY_SET_XTND_REG32((void *)(CYREG_SAR_PUMP_CTRL), regValue);
 265              		.loc 1 304 0
 266 0014 014A     		ldr	r2, .L13
 267 0016 1360     		str	r3, [r2]
 305:Generated_Source\PSoC4/cyfitter_cfg.c **** }
 268              		.loc 1 305 0
 269              		@ sp needed
 270 0018 7047     		bx	lr
 271              	.L14:
 272 001a C046     		.align	2
 273              	.L13:
 274 001c 80031A40 		.word	1075446656
 275              		.cfi_endproc
 276              	.LFE6:
 277              		.size	SetAnalogRoutingPumps, .-SetAnalogRoutingPumps
 278              		.section	.text.AnalogSetDefault,"ax",%progbits
 279              		.align	2
 280              		.code	16
 281              		.thumb_func
 282              		.type	AnalogSetDefault, %function
 283              	AnalogSetDefault:
 284              	.LFB5:
 271:Generated_Source\PSoC4/cyfitter_cfg.c **** 	CY_SET_XTND_REG32((void CYFAR *)CYREG_SAR_MUX_SWITCH0, 0x00040000u);
 285              		.loc 1 271 0
 286              		.cfi_startproc
 287              		@ args = 0, pretend = 0, frame = 0
 288              		@ frame_needed = 0, uses_anonymous_args = 0
 289 0000 10B5     		push	{r4, lr}
 290              		.cfi_def_cfa_offset 8
 291              		.cfi_offset 4, -8
 292              		.cfi_offset 14, -4
 272:Generated_Source\PSoC4/cyfitter_cfg.c **** 	SetAnalogRoutingPumps(1);
 293              		.loc 1 272 0
 294 0002 8022     		movs	r2, #128
 295 0004 D202     		lsls	r2, r2, #11
 296 0006 034B     		ldr	r3, .L16
 297 0008 1A60     		str	r2, [r3]
 273:Generated_Source\PSoC4/cyfitter_cfg.c **** }
 298              		.loc 1 273 0
 299 000a 0120     		movs	r0, #1
 300 000c FFF7FEFF 		bl	SetAnalogRoutingPumps
 301              	.LVL23:
 274:Generated_Source\PSoC4/cyfitter_cfg.c **** 
 302              		.loc 1 274 0
 303              		@ sp needed
 304 0010 10BD     		pop	{r4, pc}
 305              	.L17:
 306 0012 C046     		.align	2
 307              	.L16:
 308 0014 00031A40 		.word	1075446528
 309              		.cfi_endproc
 310              	.LFE5:
 311              		.size	AnalogSetDefault, .-AnalogSetDefault
 312              		.section	.text.Flex_Mux_Set,"ax",%progbits
ARM GAS  C:\Users\varun\AppData\Local\Temp\ccmQ1d3e.s 			page 12


 313              		.align	2
 314              		.global	Flex_Mux_Set
 315              		.code	16
 316              		.thumb_func
 317              		.type	Flex_Mux_Set, %function
 318              	Flex_Mux_Set:
 319              	.LFB7:
 306:Generated_Source\PSoC4/cyfitter_cfg.c **** 
 307:Generated_Source\PSoC4/cyfitter_cfg.c **** 
 308:Generated_Source\PSoC4/cyfitter_cfg.c **** #define CY_AMUX_UNUSED CYREG_CM0_ROM_DWT
 309:Generated_Source\PSoC4/cyfitter_cfg.c **** /*******************************************************************************
 310:Generated_Source\PSoC4/cyfitter_cfg.c **** * Function Name: Flex_Mux_Set
 311:Generated_Source\PSoC4/cyfitter_cfg.c **** ********************************************************************************
 312:Generated_Source\PSoC4/cyfitter_cfg.c **** * Summary:
 313:Generated_Source\PSoC4/cyfitter_cfg.c **** *  This function is used to set a particular channel as active on the AMux.
 314:Generated_Source\PSoC4/cyfitter_cfg.c **** *
 315:Generated_Source\PSoC4/cyfitter_cfg.c **** * Parameters:  
 316:Generated_Source\PSoC4/cyfitter_cfg.c **** *   channel - The mux channel input to set as active
 317:Generated_Source\PSoC4/cyfitter_cfg.c **** *
 318:Generated_Source\PSoC4/cyfitter_cfg.c **** * Return:
 319:Generated_Source\PSoC4/cyfitter_cfg.c **** *   void
 320:Generated_Source\PSoC4/cyfitter_cfg.c **** *
 321:Generated_Source\PSoC4/cyfitter_cfg.c **** *******************************************************************************/
 322:Generated_Source\PSoC4/cyfitter_cfg.c **** void Flex_Mux_Set(uint8 channel)
 323:Generated_Source\PSoC4/cyfitter_cfg.c **** {
 320              		.loc 1 323 0
 321              		.cfi_startproc
 322              		@ args = 0, pretend = 0, frame = 0
 323              		@ frame_needed = 0, uses_anonymous_args = 0
 324              		@ link register save eliminated.
 325              	.LVL24:
 324:Generated_Source\PSoC4/cyfitter_cfg.c **** 	switch (channel) {
 326              		.loc 1 324 0
 327 0000 0928     		cmp	r0, #9
 328 0002 33D8     		bhi	.L18
 329 0004 8000     		lsls	r0, r0, #2
 330              	.LVL25:
 331 0006 1A4B     		ldr	r3, .L31
 332 0008 1B58     		ldr	r3, [r3, r0]
 333 000a 9F46     		mov	pc, r3
 334              		.section	.rodata
 335              		.align	2
 336              	.L21:
 337 0000 0C000000 		.word	.L20
 338 0004 14000000 		.word	.L22
 339 0008 1C000000 		.word	.L23
 340 000c 24000000 		.word	.L24
 341 0010 2C000000 		.word	.L25
 342 0014 38000000 		.word	.L26
 343 0018 44000000 		.word	.L27
 344 001c 50000000 		.word	.L28
 345 0020 5E000000 		.word	.L29
 346 0024 66000000 		.word	.L30
 347              		.section	.text.Flex_Mux_Set
 348              	.L20:
 325:Generated_Source\PSoC4/cyfitter_cfg.c **** 		case 0u:
 326:Generated_Source\PSoC4/cyfitter_cfg.c **** 			CY_SET_REG32((void CYXDATA *)CYREG_SAR_MUX_SWITCH0, (0x40u));
ARM GAS  C:\Users\varun\AppData\Local\Temp\ccmQ1d3e.s 			page 13


 349              		.loc 1 326 0
 350 000c 4022     		movs	r2, #64
 351 000e 194B     		ldr	r3, .L31+4
 352 0010 1A60     		str	r2, [r3]
 327:Generated_Source\PSoC4/cyfitter_cfg.c **** 			break;
 353              		.loc 1 327 0
 354 0012 2BE0     		b	.L18
 355              	.L22:
 328:Generated_Source\PSoC4/cyfitter_cfg.c **** 		case 1u:
 329:Generated_Source\PSoC4/cyfitter_cfg.c **** 			CY_SET_REG32((void CYXDATA *)CYREG_SAR_MUX_SWITCH0, (0x80u));
 356              		.loc 1 329 0
 357 0014 8022     		movs	r2, #128
 358 0016 174B     		ldr	r3, .L31+4
 359 0018 1A60     		str	r2, [r3]
 330:Generated_Source\PSoC4/cyfitter_cfg.c **** 			break;
 360              		.loc 1 330 0
 361 001a 27E0     		b	.L18
 362              	.L23:
 331:Generated_Source\PSoC4/cyfitter_cfg.c **** 		case 2u:
 332:Generated_Source\PSoC4/cyfitter_cfg.c **** 			CY_SET_REG32((void CYXDATA *)CYREG_SAR_MUX_SWITCH0, (0x20u));
 363              		.loc 1 332 0
 364 001c 2022     		movs	r2, #32
 365 001e 154B     		ldr	r3, .L31+4
 366 0020 1A60     		str	r2, [r3]
 333:Generated_Source\PSoC4/cyfitter_cfg.c **** 			break;
 367              		.loc 1 333 0
 368 0022 23E0     		b	.L18
 369              	.L24:
 334:Generated_Source\PSoC4/cyfitter_cfg.c **** 		case 3u:
 335:Generated_Source\PSoC4/cyfitter_cfg.c **** 			CY_SET_REG32((void CYXDATA *)CYREG_SAR_MUX_SWITCH0, (0x10u));
 370              		.loc 1 335 0
 371 0024 1022     		movs	r2, #16
 372 0026 134B     		ldr	r3, .L31+4
 373 0028 1A60     		str	r2, [r3]
 336:Generated_Source\PSoC4/cyfitter_cfg.c **** 			break;
 374              		.loc 1 336 0
 375 002a 1FE0     		b	.L18
 376              	.L25:
 337:Generated_Source\PSoC4/cyfitter_cfg.c **** 		case 4u:
 338:Generated_Source\PSoC4/cyfitter_cfg.c **** 			CY_SET_REG32((void CYXDATA *)CYREG_HSIOM_PORT_SEL0, (CY_GET_REG32((void CYXDATA *)CYREG_HSIOM_PO
 377              		.loc 1 338 0
 378 002c 124A     		ldr	r2, .L31+8
 379 002e 1168     		ldr	r1, [r2]
 380 0030 0623     		movs	r3, #6
 381 0032 0B43     		orrs	r3, r1
 382 0034 1360     		str	r3, [r2]
 339:Generated_Source\PSoC4/cyfitter_cfg.c **** 			break;
 383              		.loc 1 339 0
 384 0036 19E0     		b	.L18
 385              	.L26:
 340:Generated_Source\PSoC4/cyfitter_cfg.c **** 		case 5u:
 341:Generated_Source\PSoC4/cyfitter_cfg.c **** 			CY_SET_REG32((void CYXDATA *)CYREG_HSIOM_PORT_SEL1, (CY_GET_REG32((void CYXDATA *)CYREG_HSIOM_PO
 386              		.loc 1 341 0
 387 0038 104A     		ldr	r2, .L31+12
 388 003a 1168     		ldr	r1, [r2]
 389 003c 6023     		movs	r3, #96
 390 003e 0B43     		orrs	r3, r1
ARM GAS  C:\Users\varun\AppData\Local\Temp\ccmQ1d3e.s 			page 14


 391 0040 1360     		str	r3, [r2]
 342:Generated_Source\PSoC4/cyfitter_cfg.c **** 			break;
 392              		.loc 1 342 0
 393 0042 13E0     		b	.L18
 394              	.L27:
 343:Generated_Source\PSoC4/cyfitter_cfg.c **** 		case 6u:
 344:Generated_Source\PSoC4/cyfitter_cfg.c **** 			CY_SET_REG32((void CYXDATA *)CYREG_HSIOM_PORT_SEL0, (CY_GET_REG32((void CYXDATA *)CYREG_HSIOM_PO
 395              		.loc 1 344 0
 396 0044 0C4A     		ldr	r2, .L31+8
 397 0046 1168     		ldr	r1, [r2]
 398 0048 6023     		movs	r3, #96
 399 004a 0B43     		orrs	r3, r1
 400 004c 1360     		str	r3, [r2]
 345:Generated_Source\PSoC4/cyfitter_cfg.c **** 			break;
 401              		.loc 1 345 0
 402 004e 0DE0     		b	.L18
 403              	.L28:
 346:Generated_Source\PSoC4/cyfitter_cfg.c **** 		case 7u:
 347:Generated_Source\PSoC4/cyfitter_cfg.c **** 			CY_SET_REG32((void CYXDATA *)CYREG_HSIOM_PORT_SEL1, (CY_GET_REG32((void CYXDATA *)CYREG_HSIOM_PO
 404              		.loc 1 347 0
 405 0050 0A4A     		ldr	r2, .L31+12
 406 0052 1368     		ldr	r3, [r2]
 407 0054 C021     		movs	r1, #192
 408 0056 C900     		lsls	r1, r1, #3
 409 0058 0B43     		orrs	r3, r1
 410 005a 1360     		str	r3, [r2]
 348:Generated_Source\PSoC4/cyfitter_cfg.c **** 			break;
 411              		.loc 1 348 0
 412 005c 06E0     		b	.L18
 413              	.L29:
 349:Generated_Source\PSoC4/cyfitter_cfg.c **** 		case 8u:
 350:Generated_Source\PSoC4/cyfitter_cfg.c **** 			CY_SET_REG32((void CYXDATA *)CYREG_SAR_MUX_SWITCH0, (0x04u));
 414              		.loc 1 350 0
 415 005e 0422     		movs	r2, #4
 416 0060 044B     		ldr	r3, .L31+4
 417 0062 1A60     		str	r2, [r3]
 351:Generated_Source\PSoC4/cyfitter_cfg.c **** 			break;
 418              		.loc 1 351 0
 419 0064 02E0     		b	.L18
 420              	.L30:
 352:Generated_Source\PSoC4/cyfitter_cfg.c **** 		case 9u:
 353:Generated_Source\PSoC4/cyfitter_cfg.c **** 			CY_SET_REG32((void CYXDATA *)CYREG_SAR_MUX_SWITCH0, (0x08u));
 421              		.loc 1 353 0
 422 0066 0822     		movs	r2, #8
 423 0068 024B     		ldr	r3, .L31+4
 424 006a 1A60     		str	r2, [r3]
 425              	.L18:
 354:Generated_Source\PSoC4/cyfitter_cfg.c **** 			break;
 355:Generated_Source\PSoC4/cyfitter_cfg.c **** 		default:
 356:Generated_Source\PSoC4/cyfitter_cfg.c **** 			break;
 357:Generated_Source\PSoC4/cyfitter_cfg.c **** 	}
 358:Generated_Source\PSoC4/cyfitter_cfg.c **** }
 426              		.loc 1 358 0
 427              		@ sp needed
 428 006c 7047     		bx	lr
 429              	.L32:
 430 006e C046     		.align	2
ARM GAS  C:\Users\varun\AppData\Local\Temp\ccmQ1d3e.s 			page 15


 431              	.L31:
 432 0070 00000000 		.word	.L21
 433 0074 00031A40 		.word	1075446528
 434 0078 00000140 		.word	1073807360
 435 007c 04000140 		.word	1073807364
 436              		.cfi_endproc
 437              	.LFE7:
 438              		.size	Flex_Mux_Set, .-Flex_Mux_Set
 439              		.section	.text.Flex_Mux_Unset,"ax",%progbits
 440              		.align	2
 441              		.global	Flex_Mux_Unset
 442              		.code	16
 443              		.thumb_func
 444              		.type	Flex_Mux_Unset, %function
 445              	Flex_Mux_Unset:
 446              	.LFB8:
 359:Generated_Source\PSoC4/cyfitter_cfg.c **** 
 360:Generated_Source\PSoC4/cyfitter_cfg.c **** /*******************************************************************************
 361:Generated_Source\PSoC4/cyfitter_cfg.c **** * Function Name: Flex_Mux_Unset
 362:Generated_Source\PSoC4/cyfitter_cfg.c **** ********************************************************************************
 363:Generated_Source\PSoC4/cyfitter_cfg.c **** * Summary:
 364:Generated_Source\PSoC4/cyfitter_cfg.c **** *  This function is used to clear a particular channel from being active on the
 365:Generated_Source\PSoC4/cyfitter_cfg.c **** *  AMux.
 366:Generated_Source\PSoC4/cyfitter_cfg.c **** *
 367:Generated_Source\PSoC4/cyfitter_cfg.c **** * Parameters:  
 368:Generated_Source\PSoC4/cyfitter_cfg.c **** *   channel - The mux channel input to mark inactive
 369:Generated_Source\PSoC4/cyfitter_cfg.c **** *
 370:Generated_Source\PSoC4/cyfitter_cfg.c **** * Return:
 371:Generated_Source\PSoC4/cyfitter_cfg.c **** *   void
 372:Generated_Source\PSoC4/cyfitter_cfg.c **** *
 373:Generated_Source\PSoC4/cyfitter_cfg.c **** *******************************************************************************/
 374:Generated_Source\PSoC4/cyfitter_cfg.c **** void Flex_Mux_Unset(uint8 channel)
 375:Generated_Source\PSoC4/cyfitter_cfg.c **** {
 447              		.loc 1 375 0
 448              		.cfi_startproc
 449              		@ args = 0, pretend = 0, frame = 0
 450              		@ frame_needed = 0, uses_anonymous_args = 0
 451              		@ link register save eliminated.
 452              	.LVL26:
 376:Generated_Source\PSoC4/cyfitter_cfg.c **** 	switch (channel) {
 453              		.loc 1 376 0
 454 0000 0928     		cmp	r0, #9
 455 0002 32D8     		bhi	.L33
 456 0004 8000     		lsls	r0, r0, #2
 457              	.LVL27:
 458 0006 194B     		ldr	r3, .L46
 459 0008 1B58     		ldr	r3, [r3, r0]
 460 000a 9F46     		mov	pc, r3
 461              		.section	.rodata
 462              		.align	2
 463              	.L36:
 464 0028 0C000000 		.word	.L35
 465 002c 14000000 		.word	.L37
 466 0030 1C000000 		.word	.L38
 467 0034 24000000 		.word	.L39
 468 0038 2C000000 		.word	.L40
 469 003c 38000000 		.word	.L41
ARM GAS  C:\Users\varun\AppData\Local\Temp\ccmQ1d3e.s 			page 16


 470 0040 44000000 		.word	.L42
 471 0044 50000000 		.word	.L43
 472 0048 5C000000 		.word	.L44
 473 004c 64000000 		.word	.L45
 474              		.section	.text.Flex_Mux_Unset
 475              	.L35:
 377:Generated_Source\PSoC4/cyfitter_cfg.c **** 		case 0u:
 378:Generated_Source\PSoC4/cyfitter_cfg.c **** 			CY_SET_REG32((void CYXDATA *)CYREG_SAR_MUX_SWITCH_CLEAR0, (0x40u));
 476              		.loc 1 378 0
 477 000c 4022     		movs	r2, #64
 478 000e 184B     		ldr	r3, .L46+4
 479 0010 1A60     		str	r2, [r3]
 379:Generated_Source\PSoC4/cyfitter_cfg.c **** 			break;
 480              		.loc 1 379 0
 481 0012 2AE0     		b	.L33
 482              	.L37:
 380:Generated_Source\PSoC4/cyfitter_cfg.c **** 		case 1u:
 381:Generated_Source\PSoC4/cyfitter_cfg.c **** 			CY_SET_REG32((void CYXDATA *)CYREG_SAR_MUX_SWITCH_CLEAR0, (0x80u));
 483              		.loc 1 381 0
 484 0014 8022     		movs	r2, #128
 485 0016 164B     		ldr	r3, .L46+4
 486 0018 1A60     		str	r2, [r3]
 382:Generated_Source\PSoC4/cyfitter_cfg.c **** 			break;
 487              		.loc 1 382 0
 488 001a 26E0     		b	.L33
 489              	.L38:
 383:Generated_Source\PSoC4/cyfitter_cfg.c **** 		case 2u:
 384:Generated_Source\PSoC4/cyfitter_cfg.c **** 			CY_SET_REG32((void CYXDATA *)CYREG_SAR_MUX_SWITCH_CLEAR0, (0x20u));
 490              		.loc 1 384 0
 491 001c 2022     		movs	r2, #32
 492 001e 144B     		ldr	r3, .L46+4
 493 0020 1A60     		str	r2, [r3]
 385:Generated_Source\PSoC4/cyfitter_cfg.c **** 			break;
 494              		.loc 1 385 0
 495 0022 22E0     		b	.L33
 496              	.L39:
 386:Generated_Source\PSoC4/cyfitter_cfg.c **** 		case 3u:
 387:Generated_Source\PSoC4/cyfitter_cfg.c **** 			CY_SET_REG32((void CYXDATA *)CYREG_SAR_MUX_SWITCH_CLEAR0, (0x10u));
 497              		.loc 1 387 0
 498 0024 1022     		movs	r2, #16
 499 0026 124B     		ldr	r3, .L46+4
 500 0028 1A60     		str	r2, [r3]
 388:Generated_Source\PSoC4/cyfitter_cfg.c **** 			break;
 501              		.loc 1 388 0
 502 002a 1EE0     		b	.L33
 503              	.L40:
 389:Generated_Source\PSoC4/cyfitter_cfg.c **** 		case 4u:
 390:Generated_Source\PSoC4/cyfitter_cfg.c **** 			CY_SET_REG32((void CYXDATA *)CYREG_HSIOM_PORT_SEL0, (CY_GET_REG32((void CYXDATA *)CYREG_HSIOM_PO
 504              		.loc 1 390 0
 505 002c 114A     		ldr	r2, .L46+8
 506 002e 1368     		ldr	r3, [r2]
 507 0030 0621     		movs	r1, #6
 508 0032 8B43     		bics	r3, r1
 509 0034 1360     		str	r3, [r2]
 391:Generated_Source\PSoC4/cyfitter_cfg.c **** 			break;
 510              		.loc 1 391 0
 511 0036 18E0     		b	.L33
ARM GAS  C:\Users\varun\AppData\Local\Temp\ccmQ1d3e.s 			page 17


 512              	.L41:
 392:Generated_Source\PSoC4/cyfitter_cfg.c **** 		case 5u:
 393:Generated_Source\PSoC4/cyfitter_cfg.c **** 			CY_SET_REG32((void CYXDATA *)CYREG_HSIOM_PORT_SEL1, (CY_GET_REG32((void CYXDATA *)CYREG_HSIOM_PO
 513              		.loc 1 393 0
 514 0038 0F4A     		ldr	r2, .L46+12
 515 003a 1368     		ldr	r3, [r2]
 516 003c 6021     		movs	r1, #96
 517 003e 8B43     		bics	r3, r1
 518 0040 1360     		str	r3, [r2]
 394:Generated_Source\PSoC4/cyfitter_cfg.c **** 			break;
 519              		.loc 1 394 0
 520 0042 12E0     		b	.L33
 521              	.L42:
 395:Generated_Source\PSoC4/cyfitter_cfg.c **** 		case 6u:
 396:Generated_Source\PSoC4/cyfitter_cfg.c **** 			CY_SET_REG32((void CYXDATA *)CYREG_HSIOM_PORT_SEL0, (CY_GET_REG32((void CYXDATA *)CYREG_HSIOM_PO
 522              		.loc 1 396 0
 523 0044 0B4A     		ldr	r2, .L46+8
 524 0046 1368     		ldr	r3, [r2]
 525 0048 6021     		movs	r1, #96
 526 004a 8B43     		bics	r3, r1
 527 004c 1360     		str	r3, [r2]
 397:Generated_Source\PSoC4/cyfitter_cfg.c **** 			break;
 528              		.loc 1 397 0
 529 004e 0CE0     		b	.L33
 530              	.L43:
 398:Generated_Source\PSoC4/cyfitter_cfg.c **** 		case 7u:
 399:Generated_Source\PSoC4/cyfitter_cfg.c **** 			CY_SET_REG32((void CYXDATA *)CYREG_HSIOM_PORT_SEL1, (CY_GET_REG32((void CYXDATA *)CYREG_HSIOM_PO
 531              		.loc 1 399 0
 532 0050 094A     		ldr	r2, .L46+12
 533 0052 1168     		ldr	r1, [r2]
 534 0054 094B     		ldr	r3, .L46+16
 535 0056 0B40     		ands	r3, r1
 536 0058 1360     		str	r3, [r2]
 400:Generated_Source\PSoC4/cyfitter_cfg.c **** 			break;
 537              		.loc 1 400 0
 538 005a 06E0     		b	.L33
 539              	.L44:
 401:Generated_Source\PSoC4/cyfitter_cfg.c **** 		case 8u:
 402:Generated_Source\PSoC4/cyfitter_cfg.c **** 			CY_SET_REG32((void CYXDATA *)CYREG_SAR_MUX_SWITCH_CLEAR0, (0x04u));
 540              		.loc 1 402 0
 541 005c 0422     		movs	r2, #4
 542 005e 044B     		ldr	r3, .L46+4
 543 0060 1A60     		str	r2, [r3]
 403:Generated_Source\PSoC4/cyfitter_cfg.c **** 			break;
 544              		.loc 1 403 0
 545 0062 02E0     		b	.L33
 546              	.L45:
 404:Generated_Source\PSoC4/cyfitter_cfg.c **** 		case 9u:
 405:Generated_Source\PSoC4/cyfitter_cfg.c **** 			CY_SET_REG32((void CYXDATA *)CYREG_SAR_MUX_SWITCH_CLEAR0, (0x08u));
 547              		.loc 1 405 0
 548 0064 0822     		movs	r2, #8
 549 0066 024B     		ldr	r3, .L46+4
 550 0068 1A60     		str	r2, [r3]
 551              	.L33:
 406:Generated_Source\PSoC4/cyfitter_cfg.c **** 			break;
 407:Generated_Source\PSoC4/cyfitter_cfg.c **** 		default:
 408:Generated_Source\PSoC4/cyfitter_cfg.c **** 			break;
ARM GAS  C:\Users\varun\AppData\Local\Temp\ccmQ1d3e.s 			page 18


 409:Generated_Source\PSoC4/cyfitter_cfg.c **** 	}
 410:Generated_Source\PSoC4/cyfitter_cfg.c **** }
 552              		.loc 1 410 0
 553              		@ sp needed
 554 006a 7047     		bx	lr
 555              	.L47:
 556              		.align	2
 557              	.L46:
 558 006c 28000000 		.word	.L36
 559 0070 04031A40 		.word	1075446532
 560 0074 00000140 		.word	1073807360
 561 0078 04000140 		.word	1073807364
 562 007c FFF9FFFF 		.word	-1537
 563              		.cfi_endproc
 564              	.LFE8:
 565              		.size	Flex_Mux_Unset, .-Flex_Mux_Unset
 566              		.section	.psocinit
 567              		.align	2
 568              		.global	cyfitter_cfg
 569              		.code	16
 570              		.thumb_func
 571              		.type	cyfitter_cfg, %function
 572              	cyfitter_cfg:
 573              	.LFB9:
 411:Generated_Source\PSoC4/cyfitter_cfg.c **** 
 412:Generated_Source\PSoC4/cyfitter_cfg.c **** 
 413:Generated_Source\PSoC4/cyfitter_cfg.c **** 
 414:Generated_Source\PSoC4/cyfitter_cfg.c **** /*******************************************************************************
 415:Generated_Source\PSoC4/cyfitter_cfg.c **** * Function Name: cyfitter_cfg
 416:Generated_Source\PSoC4/cyfitter_cfg.c **** ********************************************************************************
 417:Generated_Source\PSoC4/cyfitter_cfg.c **** * Summary:
 418:Generated_Source\PSoC4/cyfitter_cfg.c **** *  This function is called by the start-up code for the selected device. It
 419:Generated_Source\PSoC4/cyfitter_cfg.c **** *  performs all of the necessary device configuration based on the design
 420:Generated_Source\PSoC4/cyfitter_cfg.c **** *  settings.  This includes settings from the Design Wide Resources (DWR) such
 421:Generated_Source\PSoC4/cyfitter_cfg.c **** *  as Clocks and Pins as well as any component configuration that is necessary.
 422:Generated_Source\PSoC4/cyfitter_cfg.c **** *
 423:Generated_Source\PSoC4/cyfitter_cfg.c **** * Parameters:
 424:Generated_Source\PSoC4/cyfitter_cfg.c **** *   void
 425:Generated_Source\PSoC4/cyfitter_cfg.c **** *
 426:Generated_Source\PSoC4/cyfitter_cfg.c **** * Return:
 427:Generated_Source\PSoC4/cyfitter_cfg.c **** *   void
 428:Generated_Source\PSoC4/cyfitter_cfg.c **** *
 429:Generated_Source\PSoC4/cyfitter_cfg.c **** *******************************************************************************/
 430:Generated_Source\PSoC4/cyfitter_cfg.c **** CY_CFG_SECTION
 431:Generated_Source\PSoC4/cyfitter_cfg.c **** void cyfitter_cfg(void)
 432:Generated_Source\PSoC4/cyfitter_cfg.c **** {
 574              		.loc 1 432 0
 575              		.cfi_startproc
 576              		@ args = 0, pretend = 0, frame = 0
 577              		@ frame_needed = 0, uses_anonymous_args = 0
 578 00a8 10B5     		push	{r4, lr}
 579              		.cfi_def_cfa_offset 8
 580              		.cfi_offset 4, -8
 581              		.cfi_offset 14, -4
 433:Generated_Source\PSoC4/cyfitter_cfg.c **** 	/* Disable interrupts by default. Let user enable if/when they want. */
 434:Generated_Source\PSoC4/cyfitter_cfg.c **** 	CyGlobalIntDisable;
 582              		.loc 1 434 0
ARM GAS  C:\Users\varun\AppData\Local\Temp\ccmQ1d3e.s 			page 19


 583              		.syntax divided
 584              	@ 434 "Generated_Source\PSoC4\cyfitter_cfg.c" 1
 585 00aa 72B6     		CPSID   i
 586              	@ 0 "" 2
 435:Generated_Source\PSoC4/cyfitter_cfg.c **** 
 436:Generated_Source\PSoC4/cyfitter_cfg.c **** 	/* Enable the clock in the interrupt controller for the routed interrupts */
 437:Generated_Source\PSoC4/cyfitter_cfg.c **** 	CY_SET_REG8((void *)CYREG_UDB_UDBIF_INT_CLK_CTL, 0x01u);
 587              		.loc 1 437 0
 588              		.thumb
 589              		.syntax unified
 590 00ac 0122     		movs	r2, #1
 591 00ae 344B     		ldr	r3, .L51
 592 00b0 1A70     		strb	r2, [r3]
 593              	.LVL28:
 594              	.LBB3:
 438:Generated_Source\PSoC4/cyfitter_cfg.c **** 	{
 439:Generated_Source\PSoC4/cyfitter_cfg.c **** 		static const uint32 CYCODE cy_cfg_addr_table[] = {
 440:Generated_Source\PSoC4/cyfitter_cfg.c **** 			0x400F0001u, /* Base address: 0x400F0000 Count: 1 */
 441:Generated_Source\PSoC4/cyfitter_cfg.c **** 			0x400F3004u, /* Base address: 0x400F3000 Count: 4 */
 442:Generated_Source\PSoC4/cyfitter_cfg.c **** 			0x400F3102u, /* Base address: 0x400F3100 Count: 2 */
 443:Generated_Source\PSoC4/cyfitter_cfg.c **** 			0x400F3230u, /* Base address: 0x400F3200 Count: 48 */
 444:Generated_Source\PSoC4/cyfitter_cfg.c **** 			0x400F3316u, /* Base address: 0x400F3300 Count: 22 */
 445:Generated_Source\PSoC4/cyfitter_cfg.c **** 			0x400F4006u, /* Base address: 0x400F4000 Count: 6 */
 446:Generated_Source\PSoC4/cyfitter_cfg.c **** 			0x400F4105u, /* Base address: 0x400F4100 Count: 5 */
 447:Generated_Source\PSoC4/cyfitter_cfg.c **** 			0x400F6002u, /* Base address: 0x400F6000 Count: 2 */
 448:Generated_Source\PSoC4/cyfitter_cfg.c **** 		};
 449:Generated_Source\PSoC4/cyfitter_cfg.c **** 
 450:Generated_Source\PSoC4/cyfitter_cfg.c **** 		static const cy_cfg_addrvalue_t CYCODE cy_cfg_data_table[] = {
 451:Generated_Source\PSoC4/cyfitter_cfg.c **** 			{0x83u, 0x0Du},
 452:Generated_Source\PSoC4/cyfitter_cfg.c **** 			{0xB6u, 0x01u},
 453:Generated_Source\PSoC4/cyfitter_cfg.c **** 			{0xBEu, 0x40u},
 454:Generated_Source\PSoC4/cyfitter_cfg.c **** 			{0xD8u, 0x04u},
 455:Generated_Source\PSoC4/cyfitter_cfg.c **** 			{0xDFu, 0x01u},
 456:Generated_Source\PSoC4/cyfitter_cfg.c **** 			{0x1Fu, 0x80u},
 457:Generated_Source\PSoC4/cyfitter_cfg.c **** 			{0x83u, 0x08u},
 458:Generated_Source\PSoC4/cyfitter_cfg.c **** 			{0x40u, 0x45u},
 459:Generated_Source\PSoC4/cyfitter_cfg.c **** 			{0x49u, 0xFFu},
 460:Generated_Source\PSoC4/cyfitter_cfg.c **** 			{0x4Au, 0xFFu},
 461:Generated_Source\PSoC4/cyfitter_cfg.c **** 			{0x4Bu, 0xFFu},
 462:Generated_Source\PSoC4/cyfitter_cfg.c **** 			{0x4Fu, 0x01u},
 463:Generated_Source\PSoC4/cyfitter_cfg.c **** 			{0x50u, 0x18u},
 464:Generated_Source\PSoC4/cyfitter_cfg.c **** 			{0x5Au, 0x04u},
 465:Generated_Source\PSoC4/cyfitter_cfg.c **** 			{0x5Fu, 0x01u},
 466:Generated_Source\PSoC4/cyfitter_cfg.c **** 			{0x60u, 0x40u},
 467:Generated_Source\PSoC4/cyfitter_cfg.c **** 			{0x62u, 0x40u},
 468:Generated_Source\PSoC4/cyfitter_cfg.c **** 			{0x64u, 0x40u},
 469:Generated_Source\PSoC4/cyfitter_cfg.c **** 			{0x65u, 0x40u},
 470:Generated_Source\PSoC4/cyfitter_cfg.c **** 			{0x66u, 0x80u},
 471:Generated_Source\PSoC4/cyfitter_cfg.c **** 			{0x68u, 0x80u},
 472:Generated_Source\PSoC4/cyfitter_cfg.c **** 			{0x6Au, 0x80u},
 473:Generated_Source\PSoC4/cyfitter_cfg.c **** 			{0x6Cu, 0x80u},
 474:Generated_Source\PSoC4/cyfitter_cfg.c **** 			{0x6Eu, 0x80u},
 475:Generated_Source\PSoC4/cyfitter_cfg.c **** 			{0x8Eu, 0x01u},
 476:Generated_Source\PSoC4/cyfitter_cfg.c **** 			{0x92u, 0x01u},
 477:Generated_Source\PSoC4/cyfitter_cfg.c **** 			{0xB0u, 0x01u},
 478:Generated_Source\PSoC4/cyfitter_cfg.c **** 			{0xB2u, 0x01u},
 479:Generated_Source\PSoC4/cyfitter_cfg.c **** 			{0xBEu, 0x01u},
ARM GAS  C:\Users\varun\AppData\Local\Temp\ccmQ1d3e.s 			page 20


 480:Generated_Source\PSoC4/cyfitter_cfg.c **** 			{0xC0u, 0x54u},
 481:Generated_Source\PSoC4/cyfitter_cfg.c **** 			{0xC5u, 0xECu},
 482:Generated_Source\PSoC4/cyfitter_cfg.c **** 			{0xC7u, 0x20u},
 483:Generated_Source\PSoC4/cyfitter_cfg.c **** 			{0xC8u, 0x23u},
 484:Generated_Source\PSoC4/cyfitter_cfg.c **** 			{0xC9u, 0xFFu},
 485:Generated_Source\PSoC4/cyfitter_cfg.c **** 			{0xCAu, 0xFFu},
 486:Generated_Source\PSoC4/cyfitter_cfg.c **** 			{0xCBu, 0xFFu},
 487:Generated_Source\PSoC4/cyfitter_cfg.c **** 			{0xCDu, 0x83u},
 488:Generated_Source\PSoC4/cyfitter_cfg.c **** 			{0xCEu, 0x03u},
 489:Generated_Source\PSoC4/cyfitter_cfg.c **** 			{0xCFu, 0x01u},
 490:Generated_Source\PSoC4/cyfitter_cfg.c **** 			{0xD0u, 0x18u},
 491:Generated_Source\PSoC4/cyfitter_cfg.c **** 			{0xD2u, 0x80u},
 492:Generated_Source\PSoC4/cyfitter_cfg.c **** 			{0xD4u, 0x01u},
 493:Generated_Source\PSoC4/cyfitter_cfg.c **** 			{0xD8u, 0x04u},
 494:Generated_Source\PSoC4/cyfitter_cfg.c **** 			{0xDAu, 0x04u},
 495:Generated_Source\PSoC4/cyfitter_cfg.c **** 			{0xDBu, 0x04u},
 496:Generated_Source\PSoC4/cyfitter_cfg.c **** 			{0xDFu, 0x01u},
 497:Generated_Source\PSoC4/cyfitter_cfg.c **** 			{0xE0u, 0x40u},
 498:Generated_Source\PSoC4/cyfitter_cfg.c **** 			{0xE2u, 0x40u},
 499:Generated_Source\PSoC4/cyfitter_cfg.c **** 			{0xE4u, 0x40u},
 500:Generated_Source\PSoC4/cyfitter_cfg.c **** 			{0xE5u, 0x40u},
 501:Generated_Source\PSoC4/cyfitter_cfg.c **** 			{0xE6u, 0x80u},
 502:Generated_Source\PSoC4/cyfitter_cfg.c **** 			{0xE8u, 0x80u},
 503:Generated_Source\PSoC4/cyfitter_cfg.c **** 			{0xEAu, 0x80u},
 504:Generated_Source\PSoC4/cyfitter_cfg.c **** 			{0xECu, 0x80u},
 505:Generated_Source\PSoC4/cyfitter_cfg.c **** 			{0xEEu, 0x80u},
 506:Generated_Source\PSoC4/cyfitter_cfg.c **** 			{0x02u, 0x02u},
 507:Generated_Source\PSoC4/cyfitter_cfg.c **** 			{0x0Bu, 0x40u},
 508:Generated_Source\PSoC4/cyfitter_cfg.c **** 			{0x1Au, 0x40u},
 509:Generated_Source\PSoC4/cyfitter_cfg.c **** 			{0x1Bu, 0x08u},
 510:Generated_Source\PSoC4/cyfitter_cfg.c **** 			{0x41u, 0x01u},
 511:Generated_Source\PSoC4/cyfitter_cfg.c **** 			{0x46u, 0x80u},
 512:Generated_Source\PSoC4/cyfitter_cfg.c **** 			{0x49u, 0x05u},
 513:Generated_Source\PSoC4/cyfitter_cfg.c **** 			{0x4Bu, 0x40u},
 514:Generated_Source\PSoC4/cyfitter_cfg.c **** 			{0x4Eu, 0x02u},
 515:Generated_Source\PSoC4/cyfitter_cfg.c **** 			{0x51u, 0x01u},
 516:Generated_Source\PSoC4/cyfitter_cfg.c **** 			{0x52u, 0x02u},
 517:Generated_Source\PSoC4/cyfitter_cfg.c **** 			{0x59u, 0x05u},
 518:Generated_Source\PSoC4/cyfitter_cfg.c **** 			{0x5Au, 0x40u},
 519:Generated_Source\PSoC4/cyfitter_cfg.c **** 			{0x72u, 0x80u},
 520:Generated_Source\PSoC4/cyfitter_cfg.c **** 			{0x73u, 0x40u},
 521:Generated_Source\PSoC4/cyfitter_cfg.c **** 			{0xA7u, 0x08u},
 522:Generated_Source\PSoC4/cyfitter_cfg.c **** 			{0xAFu, 0x80u},
 523:Generated_Source\PSoC4/cyfitter_cfg.c **** 			{0xC0u, 0x01u},
 524:Generated_Source\PSoC4/cyfitter_cfg.c **** 			{0xC2u, 0x08u},
 525:Generated_Source\PSoC4/cyfitter_cfg.c **** 			{0xD0u, 0x81u},
 526:Generated_Source\PSoC4/cyfitter_cfg.c **** 			{0xD2u, 0x18u},
 527:Generated_Source\PSoC4/cyfitter_cfg.c **** 			{0xD6u, 0x0Bu},
 528:Generated_Source\PSoC4/cyfitter_cfg.c **** 			{0x57u, 0x20u},
 529:Generated_Source\PSoC4/cyfitter_cfg.c **** 			{0x6Cu, 0x04u},
 530:Generated_Source\PSoC4/cyfitter_cfg.c **** 			{0x80u, 0x04u},
 531:Generated_Source\PSoC4/cyfitter_cfg.c **** 			{0xD4u, 0x40u},
 532:Generated_Source\PSoC4/cyfitter_cfg.c **** 			{0xDAu, 0x80u},
 533:Generated_Source\PSoC4/cyfitter_cfg.c **** 			{0xE6u, 0x80u},
 534:Generated_Source\PSoC4/cyfitter_cfg.c **** 			{0x57u, 0x01u},
 535:Generated_Source\PSoC4/cyfitter_cfg.c **** 			{0xA3u, 0x01u},
 536:Generated_Source\PSoC4/cyfitter_cfg.c **** 			{0xAFu, 0x21u},
ARM GAS  C:\Users\varun\AppData\Local\Temp\ccmQ1d3e.s 			page 21


 537:Generated_Source\PSoC4/cyfitter_cfg.c **** 			{0xD6u, 0x20u},
 538:Generated_Source\PSoC4/cyfitter_cfg.c **** 			{0xEEu, 0x10u},
 539:Generated_Source\PSoC4/cyfitter_cfg.c **** 			{0x01u, 0x01u},
 540:Generated_Source\PSoC4/cyfitter_cfg.c **** 			{0x10u, 0x01u},
 541:Generated_Source\PSoC4/cyfitter_cfg.c **** 		};
 542:Generated_Source\PSoC4/cyfitter_cfg.c **** 
 543:Generated_Source\PSoC4/cyfitter_cfg.c **** 
 544:Generated_Source\PSoC4/cyfitter_cfg.c **** 
 545:Generated_Source\PSoC4/cyfitter_cfg.c **** 		CYPACKED typedef struct {
 546:Generated_Source\PSoC4/cyfitter_cfg.c **** 			void CYFAR *address;
 547:Generated_Source\PSoC4/cyfitter_cfg.c **** 			uint16 size;
 548:Generated_Source\PSoC4/cyfitter_cfg.c **** 		} CYPACKED_ATTR cfg_memset_t;
 549:Generated_Source\PSoC4/cyfitter_cfg.c **** 
 550:Generated_Source\PSoC4/cyfitter_cfg.c **** 		static const cfg_memset_t CYCODE cfg_memset_list[] = {
 551:Generated_Source\PSoC4/cyfitter_cfg.c **** 			/* address, size */
 552:Generated_Source\PSoC4/cyfitter_cfg.c **** 			{(void CYFAR *)(CYDEV_UDB_P0_U0_BASE), 1024u},
 553:Generated_Source\PSoC4/cyfitter_cfg.c **** 			{(void CYFAR *)(CYDEV_UDB_DSI0_BASE), 1024u},
 554:Generated_Source\PSoC4/cyfitter_cfg.c **** 		};
 555:Generated_Source\PSoC4/cyfitter_cfg.c **** 
 556:Generated_Source\PSoC4/cyfitter_cfg.c **** 		uint8 CYDATA i;
 557:Generated_Source\PSoC4/cyfitter_cfg.c **** 
 558:Generated_Source\PSoC4/cyfitter_cfg.c **** 		/* Zero out critical memory blocks before beginning configuration */
 559:Generated_Source\PSoC4/cyfitter_cfg.c **** 		for (i = 0u; i < (sizeof(cfg_memset_list)/sizeof(cfg_memset_list[0])); i++)
 595              		.loc 1 559 0
 596 00b2 0024     		movs	r4, #0
 597 00b4 0FE0     		b	.L49
 598              	.LVL29:
 599              	.L50:
 600              	.LBB4:
 560:Generated_Source\PSoC4/cyfitter_cfg.c **** 		{
 561:Generated_Source\PSoC4/cyfitter_cfg.c **** 			const cfg_memset_t CYCODE * CYDATA ms = &cfg_memset_list[i];
 562:Generated_Source\PSoC4/cyfitter_cfg.c **** 			CYMEMZERO(ms->address, (size_t)(uint32)(ms->size));
 601              		.loc 1 562 0 discriminator 3
 602 00b6 3348     		ldr	r0, .L51+4
 603 00b8 6200     		lsls	r2, r4, #1
 604 00ba 1319     		adds	r3, r2, r4
 605 00bc 5900     		lsls	r1, r3, #1
 606 00be 0B00     		movs	r3, r1
 607 00c0 4118     		adds	r1, r0, r1
 608 00c2 8988     		ldrh	r1, [r1, #4]
 609 00c4 1A5A     		ldrh	r2, [r3, r0]
 610 00c6 C318     		adds	r3, r0, r3
 611 00c8 5888     		ldrh	r0, [r3, #2]
 612 00ca 0004     		lsls	r0, r0, #16
 613 00cc 1043     		orrs	r0, r2
 614 00ce FFF7FEFF 		bl	CYMEMZERO
 615              	.LVL30:
 616              	.LBE4:
 559:Generated_Source\PSoC4/cyfitter_cfg.c **** 		{
 617              		.loc 1 559 0 discriminator 3
 618 00d2 0134     		adds	r4, r4, #1
 619              	.LVL31:
 620 00d4 E4B2     		uxtb	r4, r4
 621              	.LVL32:
 622              	.L49:
 559:Generated_Source\PSoC4/cyfitter_cfg.c **** 		{
 623              		.loc 1 559 0 is_stmt 0 discriminator 1
ARM GAS  C:\Users\varun\AppData\Local\Temp\ccmQ1d3e.s 			page 22


 624 00d6 012C     		cmp	r4, #1
 625 00d8 EDD9     		bls	.L50
 563:Generated_Source\PSoC4/cyfitter_cfg.c **** 		}
 564:Generated_Source\PSoC4/cyfitter_cfg.c **** 
 565:Generated_Source\PSoC4/cyfitter_cfg.c **** 		cfg_write_bytes32(cy_cfg_addr_table, cy_cfg_data_table);
 626              		.loc 1 565 0 is_stmt 1
 627 00da 2A49     		ldr	r1, .L51+4
 628 00dc 0C31     		adds	r1, r1, #12
 629 00de 2A48     		ldr	r0, .L51+8
 630 00e0 4030     		adds	r0, r0, #64
 631 00e2 FFF7FEFF 		bl	cfg_write_bytes32
 632              	.LVL33:
 566:Generated_Source\PSoC4/cyfitter_cfg.c **** 
 567:Generated_Source\PSoC4/cyfitter_cfg.c **** 		/* HSIOM Starting address: CYDEV_HSIOM_BASE */
 568:Generated_Source\PSoC4/cyfitter_cfg.c **** 		CY_SET_REG32((void *)(CYREG_HSIOM_PORT_SEL3), 0x0000EE00u);
 633              		.loc 1 568 0
 634 00e6 EE22     		movs	r2, #238
 635 00e8 1202     		lsls	r2, r2, #8
 636 00ea 284B     		ldr	r3, .L51+12
 637 00ec 1A60     		str	r2, [r3]
 569:Generated_Source\PSoC4/cyfitter_cfg.c **** 		CY_SET_REG32((void *)(CYREG_HSIOM_PORT_SEL4), 0x000000EEu);
 638              		.loc 1 569 0
 639 00ee EE22     		movs	r2, #238
 640 00f0 274B     		ldr	r3, .L51+16
 641 00f2 1A60     		str	r2, [r3]
 570:Generated_Source\PSoC4/cyfitter_cfg.c **** 
 571:Generated_Source\PSoC4/cyfitter_cfg.c **** 		/* UDB_PA_0 Starting address: CYDEV_UDB_PA0_BASE */
 572:Generated_Source\PSoC4/cyfitter_cfg.c **** 		CY_SET_REG32((void *)(CYDEV_UDB_PA0_BASE), 0x00990000u);
 642              		.loc 1 572 0
 643 00f4 9923     		movs	r3, #153
 644 00f6 1B04     		lsls	r3, r3, #16
 645 00f8 264A     		ldr	r2, .L51+20
 646 00fa 1360     		str	r3, [r2]
 573:Generated_Source\PSoC4/cyfitter_cfg.c **** 		CY_SET_REG32((void *)(CYREG_UDB_PA0_CFG8), 0x00050000u);
 647              		.loc 1 573 0
 648 00fc A021     		movs	r1, #160
 649 00fe C902     		lsls	r1, r1, #11
 650 0100 254A     		ldr	r2, .L51+24
 651 0102 1160     		str	r1, [r2]
 574:Generated_Source\PSoC4/cyfitter_cfg.c **** 
 575:Generated_Source\PSoC4/cyfitter_cfg.c **** 		/* UDB_PA_1 Starting address: CYDEV_UDB_PA1_BASE */
 576:Generated_Source\PSoC4/cyfitter_cfg.c **** 		CY_SET_REG32((void *)(CYDEV_UDB_PA1_BASE), 0x00990000u);
 652              		.loc 1 576 0
 653 0104 254A     		ldr	r2, .L51+28
 654 0106 1360     		str	r3, [r2]
 577:Generated_Source\PSoC4/cyfitter_cfg.c **** 		CY_SET_REG32((void *)(CYREG_UDB_PA1_CFG8), 0x003C0000u);
 655              		.loc 1 577 0
 656 0108 F021     		movs	r1, #240
 657 010a 8903     		lsls	r1, r1, #14
 658 010c 244A     		ldr	r2, .L51+32
 659 010e 1160     		str	r1, [r2]
 578:Generated_Source\PSoC4/cyfitter_cfg.c **** 
 579:Generated_Source\PSoC4/cyfitter_cfg.c **** 		/* UDB_PA_2 Starting address: CYDEV_UDB_PA2_BASE */
 580:Generated_Source\PSoC4/cyfitter_cfg.c **** 		CY_SET_REG32((void *)(CYDEV_UDB_PA2_BASE), 0x00990000u);
 660              		.loc 1 580 0
 661 0110 244A     		ldr	r2, .L51+36
 662 0112 1360     		str	r3, [r2]
ARM GAS  C:\Users\varun\AppData\Local\Temp\ccmQ1d3e.s 			page 23


 581:Generated_Source\PSoC4/cyfitter_cfg.c **** 
 582:Generated_Source\PSoC4/cyfitter_cfg.c **** 		/* UDB_PA_3 Starting address: CYDEV_UDB_PA3_BASE */
 583:Generated_Source\PSoC4/cyfitter_cfg.c **** 		CY_SET_REG32((void *)(CYDEV_UDB_PA3_BASE), 0x00990000u);
 663              		.loc 1 583 0
 664 0114 244A     		ldr	r2, .L51+40
 665 0116 1360     		str	r3, [r2]
 584:Generated_Source\PSoC4/cyfitter_cfg.c **** 
 585:Generated_Source\PSoC4/cyfitter_cfg.c **** 		/* INT_SELECT Starting address: CYDEV_CPUSS_INTR_SELECT */
 586:Generated_Source\PSoC4/cyfitter_cfg.c **** 		CY_SET_REG32((void *)(CYREG_CPUSS_INTR_SELECT), 0x00000001u);
 666              		.loc 1 586 0
 667 0118 0122     		movs	r2, #1
 668 011a 244B     		ldr	r3, .L51+44
 669 011c 1A60     		str	r2, [r3]
 587:Generated_Source\PSoC4/cyfitter_cfg.c **** 
 588:Generated_Source\PSoC4/cyfitter_cfg.c **** 		/* INT_CONFIG Starting address: CYDEV_UDB_INT_CFG */
 589:Generated_Source\PSoC4/cyfitter_cfg.c **** 		CY_SET_REG32((void *)(CYREG_UDB_INT_CFG), 0x00000002u);
 670              		.loc 1 589 0
 671 011e 0221     		movs	r1, #2
 672 0120 234B     		ldr	r3, .L51+48
 673 0122 1960     		str	r1, [r3]
 590:Generated_Source\PSoC4/cyfitter_cfg.c **** 
 591:Generated_Source\PSoC4/cyfitter_cfg.c **** 		/* Enable UDB array and digital routing */
 592:Generated_Source\PSoC4/cyfitter_cfg.c **** 		CY_SET_XTND_REG8((void *)CYREG_UDB_UDBIF_WAIT_CFG, (uint8)((CY_GET_XTND_REG8((void *)CYREG_UDB_UD
 674              		.loc 1 592 0
 675 0124 2348     		ldr	r0, .L51+52
 676 0126 0378     		ldrb	r3, [r0]
 677 0128 3B32     		adds	r2, r2, #59
 678 012a 9343     		bics	r3, r2
 679 012c 1422     		movs	r2, #20
 680 012e 1343     		orrs	r3, r2
 681 0130 DBB2     		uxtb	r3, r3
 682 0132 0370     		strb	r3, [r0]
 593:Generated_Source\PSoC4/cyfitter_cfg.c **** 		CY_SET_XTND_REG8((void *)CYREG_UDB_UDBIF_BANK_CTL, (uint8)(CY_GET_XTND_REG8((void *)CYREG_UDB_UDB
 683              		.loc 1 593 0
 684 0134 204A     		ldr	r2, .L51+56
 685 0136 1078     		ldrb	r0, [r2]
 686 0138 1623     		movs	r3, #22
 687 013a 0343     		orrs	r3, r0
 688 013c DBB2     		uxtb	r3, r3
 689 013e 1370     		strb	r3, [r2]
 690              	.LBE3:
 594:Generated_Source\PSoC4/cyfitter_cfg.c **** 	}
 595:Generated_Source\PSoC4/cyfitter_cfg.c **** 
 596:Generated_Source\PSoC4/cyfitter_cfg.c **** 	/* Perform second pass device configuration. These items must be configured in specific order afte
 597:Generated_Source\PSoC4/cyfitter_cfg.c **** 	/* IOPINS0_0 Starting address: CYDEV_PRT0_BASE */
 598:Generated_Source\PSoC4/cyfitter_cfg.c **** 	CY_SET_REG32((void *)(CYDEV_PRT0_BASE), 0x00000003u);
 691              		.loc 1 598 0
 692 0140 0323     		movs	r3, #3
 693 0142 1E4A     		ldr	r2, .L51+60
 694 0144 1360     		str	r3, [r2]
 599:Generated_Source\PSoC4/cyfitter_cfg.c **** 	CY_SET_REG32((void *)(CYREG_PRT0_PC2), 0x00000003u);
 695              		.loc 1 599 0
 696 0146 1E4A     		ldr	r2, .L51+64
 697 0148 1360     		str	r3, [r2]
 600:Generated_Source\PSoC4/cyfitter_cfg.c **** 
 601:Generated_Source\PSoC4/cyfitter_cfg.c **** 	/* IOPINS0_1 Starting address: CYDEV_PRT1_BASE */
 602:Generated_Source\PSoC4/cyfitter_cfg.c **** 	CY_SET_REG32((void *)(CYDEV_PRT1_BASE), 0x00000006u);
ARM GAS  C:\Users\varun\AppData\Local\Temp\ccmQ1d3e.s 			page 24


 698              		.loc 1 602 0
 699 014a 0622     		movs	r2, #6
 700 014c 1D48     		ldr	r0, .L51+68
 701 014e 0260     		str	r2, [r0]
 603:Generated_Source\PSoC4/cyfitter_cfg.c **** 	CY_SET_REG32((void *)(CYREG_PRT1_PC2), 0x00000006u);
 702              		.loc 1 603 0
 703 0150 1D48     		ldr	r0, .L51+72
 704 0152 0260     		str	r2, [r0]
 604:Generated_Source\PSoC4/cyfitter_cfg.c **** 
 605:Generated_Source\PSoC4/cyfitter_cfg.c **** 	/* IOPINS0_2 Starting address: CYDEV_PRT2_BASE */
 606:Generated_Source\PSoC4/cyfitter_cfg.c **** 	CY_SET_REG32((void *)(CYDEV_PRT2_BASE), 0x000000FCu);
 705              		.loc 1 606 0
 706 0154 F632     		adds	r2, r2, #246
 707 0156 1D48     		ldr	r0, .L51+76
 708 0158 0260     		str	r2, [r0]
 607:Generated_Source\PSoC4/cyfitter_cfg.c **** 	CY_SET_REG32((void *)(CYREG_PRT2_PC2), 0x000000FCu);
 709              		.loc 1 607 0
 710 015a 1D48     		ldr	r0, .L51+80
 711 015c 0260     		str	r2, [r0]
 608:Generated_Source\PSoC4/cyfitter_cfg.c **** 
 609:Generated_Source\PSoC4/cyfitter_cfg.c **** 	/* IOPINS0_3 Starting address: CYDEV_PRT3_BASE */
 610:Generated_Source\PSoC4/cyfitter_cfg.c **** 	CY_SET_REG32((void *)(CYDEV_PRT3_BASE), 0x00000002u);
 712              		.loc 1 610 0
 713 015e 1D4A     		ldr	r2, .L51+84
 714 0160 1160     		str	r1, [r2]
 611:Generated_Source\PSoC4/cyfitter_cfg.c **** 	CY_SET_REG32((void *)(CYREG_PRT3_PC), 0x00000DB0u);
 715              		.loc 1 611 0
 716 0162 DB21     		movs	r1, #219
 717 0164 0901     		lsls	r1, r1, #4
 718 0166 1C4A     		ldr	r2, .L51+88
 719 0168 1160     		str	r1, [r2]
 612:Generated_Source\PSoC4/cyfitter_cfg.c **** 
 613:Generated_Source\PSoC4/cyfitter_cfg.c **** 	/* IOPINS0_4 Starting address: CYDEV_PRT4_BASE */
 614:Generated_Source\PSoC4/cyfitter_cfg.c **** 	CY_SET_REG32((void *)(CYDEV_PRT4_BASE), 0x00000003u);
 720              		.loc 1 614 0
 721 016a 1C4A     		ldr	r2, .L51+92
 722 016c 1360     		str	r3, [r2]
 615:Generated_Source\PSoC4/cyfitter_cfg.c **** 	CY_SET_REG32((void *)(CYREG_PRT4_PC), 0x00000024u);
 723              		.loc 1 615 0
 724 016e 2422     		movs	r2, #36
 725 0170 1B4B     		ldr	r3, .L51+96
 726 0172 1A60     		str	r2, [r3]
 616:Generated_Source\PSoC4/cyfitter_cfg.c **** 
 617:Generated_Source\PSoC4/cyfitter_cfg.c **** 
 618:Generated_Source\PSoC4/cyfitter_cfg.c **** 	/* Setup clocks based on selections from Clock DWR */
 619:Generated_Source\PSoC4/cyfitter_cfg.c **** 	ClockSetup();
 727              		.loc 1 619 0
 728 0174 FFF744FF 		bl	ClockSetup
 729              	.LVL34:
 620:Generated_Source\PSoC4/cyfitter_cfg.c **** 
 621:Generated_Source\PSoC4/cyfitter_cfg.c **** 	/* Perform basic analog initialization to defaults */
 622:Generated_Source\PSoC4/cyfitter_cfg.c **** 	AnalogSetDefault();
 730              		.loc 1 622 0
 731 0178 FFF7FEFF 		bl	AnalogSetDefault
 732              	.LVL35:
 623:Generated_Source\PSoC4/cyfitter_cfg.c **** 
 624:Generated_Source\PSoC4/cyfitter_cfg.c **** }
ARM GAS  C:\Users\varun\AppData\Local\Temp\ccmQ1d3e.s 			page 25


 733              		.loc 1 624 0
 734              		@ sp needed
 735              	.LVL36:
 736 017c 10BD     		pop	{r4, pc}
 737              	.L52:
 738 017e C046     		.align	2
 739              	.L51:
 740 0180 1C700F40 		.word	1074753564
 741 0184 50000000 		.word	.LANCHOR0
 742 0188 D0000000 		.word	.LANCHOR1
 743 018c 0C000140 		.word	1073807372
 744 0190 10000140 		.word	1073807376
 745 0194 00500F40 		.word	1074745344
 746 0198 08500F40 		.word	1074745352
 747 019c 10500F40 		.word	1074745360
 748 01a0 18500F40 		.word	1074745368
 749 01a4 20500F40 		.word	1074745376
 750 01a8 30500F40 		.word	1074745392
 751 01ac 20000040 		.word	1073741856
 752 01b0 00800F40 		.word	1074757632
 753 01b4 01700F40 		.word	1074753537
 754 01b8 00700F40 		.word	1074753536
 755 01bc 00000440 		.word	1074003968
 756 01c0 18000440 		.word	1074003992
 757 01c4 00010440 		.word	1074004224
 758 01c8 18010440 		.word	1074004248
 759 01cc 00020440 		.word	1074004480
 760 01d0 18020440 		.word	1074004504
 761 01d4 00030440 		.word	1074004736
 762 01d8 08030440 		.word	1074004744
 763 01dc 00040440 		.word	1074004992
 764 01e0 08040440 		.word	1074005000
 765              		.cfi_endproc
 766              	.LFE9:
 767              		.size	cyfitter_cfg, .-cyfitter_cfg
 768              		.section	.rodata
 769              		.align	2
 770              		.set	.LANCHOR0,. + 0
 771              		.set	.LANCHOR1,. + 128
 772              		.type	cfg_memset_list.4910, %object
 773              		.size	cfg_memset_list.4910, 12
 774              	cfg_memset_list.4910:
 775 0050 00300F40 		.word	1074737152
 776 0054 0004     		.short	1024
 777 0056 00400F40 		.4byte	1074741248
 778 005a 0004     		.short	1024
 779              		.type	cy_cfg_data_table.4905, %object
 780              		.size	cy_cfg_data_table.4905, 180
 781              	cy_cfg_data_table.4905:
 782 005c 83       		.byte	-125
 783 005d 0D       		.byte	13
 784 005e B6       		.byte	-74
 785 005f 01       		.byte	1
 786 0060 BE       		.byte	-66
 787 0061 40       		.byte	64
 788 0062 D8       		.byte	-40
 789 0063 04       		.byte	4
ARM GAS  C:\Users\varun\AppData\Local\Temp\ccmQ1d3e.s 			page 26


 790 0064 DF       		.byte	-33
 791 0065 01       		.byte	1
 792 0066 1F       		.byte	31
 793 0067 80       		.byte	-128
 794 0068 83       		.byte	-125
 795 0069 08       		.byte	8
 796 006a 40       		.byte	64
 797 006b 45       		.byte	69
 798 006c 49       		.byte	73
 799 006d FF       		.byte	-1
 800 006e 4A       		.byte	74
 801 006f FF       		.byte	-1
 802 0070 4B       		.byte	75
 803 0071 FF       		.byte	-1
 804 0072 4F       		.byte	79
 805 0073 01       		.byte	1
 806 0074 50       		.byte	80
 807 0075 18       		.byte	24
 808 0076 5A       		.byte	90
 809 0077 04       		.byte	4
 810 0078 5F       		.byte	95
 811 0079 01       		.byte	1
 812 007a 60       		.byte	96
 813 007b 40       		.byte	64
 814 007c 62       		.byte	98
 815 007d 40       		.byte	64
 816 007e 64       		.byte	100
 817 007f 40       		.byte	64
 818 0080 65       		.byte	101
 819 0081 40       		.byte	64
 820 0082 66       		.byte	102
 821 0083 80       		.byte	-128
 822 0084 68       		.byte	104
 823 0085 80       		.byte	-128
 824 0086 6A       		.byte	106
 825 0087 80       		.byte	-128
 826 0088 6C       		.byte	108
 827 0089 80       		.byte	-128
 828 008a 6E       		.byte	110
 829 008b 80       		.byte	-128
 830 008c 8E       		.byte	-114
 831 008d 01       		.byte	1
 832 008e 92       		.byte	-110
 833 008f 01       		.byte	1
 834 0090 B0       		.byte	-80
 835 0091 01       		.byte	1
 836 0092 B2       		.byte	-78
 837 0093 01       		.byte	1
 838 0094 BE       		.byte	-66
 839 0095 01       		.byte	1
 840 0096 C0       		.byte	-64
 841 0097 54       		.byte	84
 842 0098 C5       		.byte	-59
 843 0099 EC       		.byte	-20
 844 009a C7       		.byte	-57
 845 009b 20       		.byte	32
 846 009c C8       		.byte	-56
ARM GAS  C:\Users\varun\AppData\Local\Temp\ccmQ1d3e.s 			page 27


 847 009d 23       		.byte	35
 848 009e C9       		.byte	-55
 849 009f FF       		.byte	-1
 850 00a0 CA       		.byte	-54
 851 00a1 FF       		.byte	-1
 852 00a2 CB       		.byte	-53
 853 00a3 FF       		.byte	-1
 854 00a4 CD       		.byte	-51
 855 00a5 83       		.byte	-125
 856 00a6 CE       		.byte	-50
 857 00a7 03       		.byte	3
 858 00a8 CF       		.byte	-49
 859 00a9 01       		.byte	1
 860 00aa D0       		.byte	-48
 861 00ab 18       		.byte	24
 862 00ac D2       		.byte	-46
 863 00ad 80       		.byte	-128
 864 00ae D4       		.byte	-44
 865 00af 01       		.byte	1
 866 00b0 D8       		.byte	-40
 867 00b1 04       		.byte	4
 868 00b2 DA       		.byte	-38
 869 00b3 04       		.byte	4
 870 00b4 DB       		.byte	-37
 871 00b5 04       		.byte	4
 872 00b6 DF       		.byte	-33
 873 00b7 01       		.byte	1
 874 00b8 E0       		.byte	-32
 875 00b9 40       		.byte	64
 876 00ba E2       		.byte	-30
 877 00bb 40       		.byte	64
 878 00bc E4       		.byte	-28
 879 00bd 40       		.byte	64
 880 00be E5       		.byte	-27
 881 00bf 40       		.byte	64
 882 00c0 E6       		.byte	-26
 883 00c1 80       		.byte	-128
 884 00c2 E8       		.byte	-24
 885 00c3 80       		.byte	-128
 886 00c4 EA       		.byte	-22
 887 00c5 80       		.byte	-128
 888 00c6 EC       		.byte	-20
 889 00c7 80       		.byte	-128
 890 00c8 EE       		.byte	-18
 891 00c9 80       		.byte	-128
 892 00ca 02       		.byte	2
 893 00cb 02       		.byte	2
 894 00cc 0B       		.byte	11
 895 00cd 40       		.byte	64
 896 00ce 1A       		.byte	26
 897 00cf 40       		.byte	64
 898 00d0 1B       		.byte	27
 899 00d1 08       		.byte	8
 900 00d2 41       		.byte	65
 901 00d3 01       		.byte	1
 902 00d4 46       		.byte	70
 903 00d5 80       		.byte	-128
ARM GAS  C:\Users\varun\AppData\Local\Temp\ccmQ1d3e.s 			page 28


 904 00d6 49       		.byte	73
 905 00d7 05       		.byte	5
 906 00d8 4B       		.byte	75
 907 00d9 40       		.byte	64
 908 00da 4E       		.byte	78
 909 00db 02       		.byte	2
 910 00dc 51       		.byte	81
 911 00dd 01       		.byte	1
 912 00de 52       		.byte	82
 913 00df 02       		.byte	2
 914 00e0 59       		.byte	89
 915 00e1 05       		.byte	5
 916 00e2 5A       		.byte	90
 917 00e3 40       		.byte	64
 918 00e4 72       		.byte	114
 919 00e5 80       		.byte	-128
 920 00e6 73       		.byte	115
 921 00e7 40       		.byte	64
 922 00e8 A7       		.byte	-89
 923 00e9 08       		.byte	8
 924 00ea AF       		.byte	-81
 925 00eb 80       		.byte	-128
 926 00ec C0       		.byte	-64
 927 00ed 01       		.byte	1
 928 00ee C2       		.byte	-62
 929 00ef 08       		.byte	8
 930 00f0 D0       		.byte	-48
 931 00f1 81       		.byte	-127
 932 00f2 D2       		.byte	-46
 933 00f3 18       		.byte	24
 934 00f4 D6       		.byte	-42
 935 00f5 0B       		.byte	11
 936 00f6 57       		.byte	87
 937 00f7 20       		.byte	32
 938 00f8 6C       		.byte	108
 939 00f9 04       		.byte	4
 940 00fa 80       		.byte	-128
 941 00fb 04       		.byte	4
 942 00fc D4       		.byte	-44
 943 00fd 40       		.byte	64
 944 00fe DA       		.byte	-38
 945 00ff 80       		.byte	-128
 946 0100 E6       		.byte	-26
 947 0101 80       		.byte	-128
 948 0102 57       		.byte	87
 949 0103 01       		.byte	1
 950 0104 A3       		.byte	-93
 951 0105 01       		.byte	1
 952 0106 AF       		.byte	-81
 953 0107 21       		.byte	33
 954 0108 D6       		.byte	-42
 955 0109 20       		.byte	32
 956 010a EE       		.byte	-18
 957 010b 10       		.byte	16
 958 010c 01       		.byte	1
 959 010d 01       		.byte	1
 960 010e 10       		.byte	16
ARM GAS  C:\Users\varun\AppData\Local\Temp\ccmQ1d3e.s 			page 29


 961 010f 01       		.byte	1
 962              		.type	cy_cfg_addr_table.4904, %object
 963              		.size	cy_cfg_addr_table.4904, 32
 964              	cy_cfg_addr_table.4904:
 965 0110 01000F40 		.word	1074724865
 966 0114 04300F40 		.word	1074737156
 967 0118 02310F40 		.word	1074737410
 968 011c 30320F40 		.word	1074737712
 969 0120 16330F40 		.word	1074737942
 970 0124 06400F40 		.word	1074741254
 971 0128 05410F40 		.word	1074741509
 972 012c 02600F40 		.word	1074749442
 973              		.text
 974              	.Letext0:
 975              		.file 2 "c:\\program files (x86)\\cypress\\psoc creator\\4.4\\psoc creator\\import\\gnu\\arm\\5.4.
 976              		.file 3 "Generated_Source\\PSoC4\\cytypes.h"
 977              		.file 4 "Generated_Source\\PSoC4\\CyLib.h"
